:100000000C9407040C942F040C942F040C942F04CC
:100010000C942F040C942F040C944A370C942F0446
:100020000C942F040C942F040C942F040C942F0484
:100030000C942F040C942F040C949E380C944F397C
:100040000C942F040C942F040C942F040C942F0464
:100050000C94DB360C942F040C942F040C942F0476
:100060000C9400370C9407380C9495370C946F3728
:100070000C942F040C9491360C942F040C942F04A0
:100080000C942F040C942F040C9425370C94B63642
:100090000C942D360C94E1370C94BB370C942F0440
:1000A00007634236B79BD8A71A39685618AEBAAB61
:1000B000558C1D3CB7CC5763BD6DEDFD753EF617F5
:1000C0007231BF000000803F08000000BE9224494A
:1000D000123EABAAAA2ABECDCCCC4C3E000000807A
:1000E000BEABAAAAAA3E00000000BF000000803FED
:1000F0000000000000084178D3BB4387D1133D19AD
:100100000E3CC3BD4282AD2B3E68EC8276BED98FD9
:10011000E1A93E4C80EFFFBE01C4FF7F3F0000001D
:100120000000010008191304E81A0010191302E86E
:100130004C0011191301E8820010191301E8B400F2
:1001400011191301E8EA0010191302E81C01101933
:100150001302E84E0111191301E8000303070F3FD2
:10016000FFFF07070707070707070707070707072F
:100170000707070707E01FF83FFC7C3E700FF00FF2
:10018000E007E00700070007000F001E003C00F832
:1001900003F007C01F003C00380070006000E00062
:1001A000FFFFFFFFFFFF07F007FE07FF8783C38006
:1001B000F38039C01CE00E0007000F007F003F00F5
:1001C0001FE00078001E00070003F001F800FE00A9
:1001D000770073E0F8FFF83FF807F00000380038C8
:1001E000007800F800F801F803B8033807380E3833
:1001F0001C381838383870386038E038FFFFFFFF97
:10020000FFFF0038003800380038003800381FFF82
:100210000FFF8FFFC700038001C000E000700039AE
:10022000F03FFE1FFF8F83E700F0003C000E000749
:1002300000038001C000FC00EF0073C0F0FFF83F36
:10024000F807E00003E00FF81FFC3C1E380E700EAC
:1002500070006000E000E3E0EFF8FFFCFC3EF00E11
:10026000F00FE007E007E0076007700F700E3C3EFC
:100270003FFC1FF807E0FFFFFFFFFFFF0006000E37
:10028000001C001800380070006000E000C001C0D1
:100290000180038003800700070007000E000E00A6
:1002A0000E000C001C001C0007F00FFE0FFF8783E0
:1002B000C780F38039C01CE00E780F1E0F07FF01C6
:1002C000FF03FFE3E0F9C01DC00FE003F001F800F9
:1002D000FC00F70073E0F8FFF83FF807F000005A61
:1002E000012201310038003800000000003E5B4F61
:1002F0005B3E3E6B4F6B3E1C3E7C3E1C183C7E3C86
:10030000181C577D571C1C5E7F5E1C00183C180093
:10031000FFE7C3E7FF0018241800FFE7DBE7FF3023
:10032000483A060E2629792926407F050507407F91
:1003300005253F5A3CE73C5A7F3E1C1C08081C1C04
:100340003E7F14227F22145F5F005F5F06097F01FA
:100350007F006689956A606060606094A2FFA294E5
:1003600008047E040810207E201008082A1C0808B3
:100370001C2A08081E101010100C1E0C1E0C303801
:100380003E3830060E3E0E06000000000000005F02
:1003900000000007000700147F147F14242A7F2A1E
:1003A00012231308646236495620500008070300E0
:1003B000001C2241000041221C002A1C7F1C2A082C
:1003C000083E08080080703000080808080800008F
:1003D00060600020100804023E5149453E00427F03
:1003E000400072494949462141494D331814127F52
:1003F0001027454545393C4A4949314121110907F2
:100400003649494936464949291E00001400000072
:100410004034000000081422411414141414004144
:1004200022140802015909063E415D594E7C121101
:10043000127C7F494949363E414141227F41414139
:100440003E7F494949417F090909013E41415173B4
:100450007F0808087F00417F41002040413F017F25
:10046000081422417F404040407F021C027F7F04ED
:1004700008107F3E4141413E7F090909063E415136
:10048000215E7F09192946264949493203017F0126
:10049000033F4040403F1F2040201F3F4038403F27
:1004A000631408146303047804036159494D43003D
:1004B0007F4141410204081020004141417F040274
:1004C000010204404040404000030708002054540B
:1004D00078407F28444438384444442838444428E9
:1004E0007F385454541800087E090218A4A49C783C
:1004F0007F0804047800447D40002040403D007F98
:100500001028440000417F40007C047804787C0877
:100510000404783844444438FC182424181824244B
:1005200018FC7C08040408485454542404043F4430
:10053000243C4040207C1C2040201C3C4030403C5F
:1005400044281028444C9090907C4464544C4400BF
:100550000836410000007700000041360800020123
:100560000204023C2623263C1EA1A161123A40400F
:10057000207A38545455592155557941225454788C
:1005800042215554784020545579400C1E52721225
:1005900039555555593954545459395554545800AE
:1005A00000457C410002457D420001457C407D12B2
:1005B00011127DF0282528F07C5455450020545414
:1005C0007C547C0A097F4932494949323A444444BF
:1005D0003A324A4848303A4141217A3A42402078FA
:1005E000009DA0A07D3D4242423D3D4040403D3CFB
:1005F00024FF2424487E4943662B2FFC2F2BFF0920
:1006000029F620C0887E0903205454794100004413
:100610007D413048484A32384040227A007A0A0AFE
:10062000727D0D19317D2629292F28262929292671
:1006300030484D4020380808080808080808382FB6
:1006400010C8ACBA2F102834FA00007B0000081440
:100650002A142222142A14085500550055AA55AA16
:1006600055AAFF55FF55FF000000FF00101010FFB6
:1006700000141414FF001010FF00FF1010F010F011
:10068000141414FC001414F700FF0000FF00FF1402
:1006900014F404FC141417101F10101F101F14144E
:1006A000141F00101010F0000000001F1010101098
:1006B0001F10101010F010000000FF10101010108C
:1006C00010101010FF10000000FF140000FF00FFCA
:1006D00000001F10170000FC04F414141710171466
:1006E00014F404F40000FF00F71414141414141488
:1006F000F700F7141414171410101F101F141414FB
:10070000F4141010F010F000001F101F0000001F64
:1007100014000000FC140000F010F01010FF10FF97
:10072000141414FF141010101F00000000F010FF2C
:10073000FFFFFFFFF0F0F0F0F0FFFFFF0000000010
:1007400000FFFF0F0F0F0F0F3844443844FC4A4A94
:100750004A347E02020606027E027E026355494149
:10076000633844443C04407E201E2006027E020280
:1007700099A5E7A5991C2A492A1C4C7201724C3094
:100780004A4D4D303048784830BC625A463D3E496B
:100790004949007E0101017E2A2A2A2A2A44445F0F
:1007A000444440514A444040444A51400000FF0103
:1007B00003E080FF000008086B6B08361236243611
:1007C000060F090F06000018180000001010003076
:1007D00040FF0101001F01011E00191D1712003CFE
:1007E0003C3C3C00000000000901809611800A3A60
:1007F00081550A3601082A04000000F02B0400008D
:10080000014021800A13800A29800A000F3A11242E
:100810001FBECFEFCDBFDFE3DEBF18E2A0E0B8E23E
:10082000E3E8F1EB02C005900D92A637B107D9F7C6
:100830002EE2A6E7B8E201C01D92A431B207E1F7AB
:1008400014E0C7E0D4E004C02197FE010E94A9553E
:10085000C630D107C9F70E94A73B0C9411570C94DE
:10086000000090E0FC01EA5DF041E081EF3F39F1EA
:1008700086549041DC012C91822F880F880F880FBD
:100880008E0F8033E0F490E0880F991FDC01A75BA6
:10089000B44D6D937C938751954DDC011D921C9254
:1008A000B0E22B9FC00111249C5F4096E80FF92F06
:1008B000F11D8081887F808380818160808308959D
:1008C000CF93C82F8091C12D9091C22DDC01ED9165
:1008D000FC910688F789E02D6091C02D09958091E3
:1008E000C12D9091C22DDC01ED91FC910190F08120
:1008F000E02D6C2F09958091C12D9091C22DDC01C6
:10090000ED91FC91028CF38DE02D0995882331F057
:1009100082E88093C32D80E0CF9108958091C12D0E
:100920009091C22DDC01ED91FC91048CF58DE02DB0
:1009300021E041E050E06091C02D0995813041F700
:100940001092C32D8091C12D9091C22DDC01ED91AB
:10095000FC910284F385E02D0995DECFCF93DF93E0
:10096000D82FC62F8091C12D9091C22DDC01ED9121
:10097000FC910688F789E02D6091C02D0995809142
:10098000C12D9091C22DDC01ED91FC910190F0817F
:10099000E02D6D2F09958091C12D9091C22DDC0124
:1009A000ED91FC910190F081E02D6C2F09958091E3
:1009B000C12D9091C22DDC01ED91FC91028CF38D43
:1009C000E02D0995882339F082E88093C32D80E0DB
:1009D000DF91CF9108951092C32D81E0F9CFCF938D
:1009E000DF93D82FC62F89E00E9460049091C32D19
:1009F000911112C061E070E001C0660FDA95EAF76C
:100A0000CC2371F0682B861771F089E00E94AE0448
:100A100081E09091C32D911180E0DF91CF910895F5
:100A200060956823F0CF81E0F8CFCF93DF93D82F84
:100A3000C62F80E00E9460049091C32D911110C0D8
:100A400061E070E001C0660FDA95EAF7C23061F448
:100A5000682B80E00E94AE0481E09091C32D91113B
:100A600080E0DF91CF91089560956823F2CFFC017B
:100A700054894589252F30E0842F90E0821B930B09
:100A8000541710F0CF96089501970895FC019289AC
:100A90008389981761F0A389AE0FBF2FB11D5996B6
:100AA0008C9193899F5F9F73938B90E008958FEF54
:100AB0009FEF0895FC0192898389981731F083890B
:100AC000E80FF11D818D90E008958FEF9FEF08955D
:100AD000FC0192892389892F90E0805C9F4F821BC3
:100AE00091098F7399270895CF93DF93EC01E881E3
:100AF000F9810680F781E02D0995EC85FD858681D9
:100B00008F738683EC85FD8585818F7585838B89C1
:100B10008A8B198ADF91CF910895CF93DF93FC01DF
:100B200094898589C485D585981306C08D818F7D6C
:100B30008D83DF91CF910895A589AE0FBF2FB11D91
:100B4000A75ABF4F2C91858990E001968F73992702
:100B5000858B80E48C83A485B58512962C9394892B
:100B600085899813E6CFA485B58515968C91159740
:100B70008F7D15968C9387898823D9F2808D8093F9
:100B80001301178AD6CFDC011C96ED91FC910FB6AC
:100B900007FE03C0258125FD04C0248125FD0C949A
:100BA0008D050895EF92FF920F931F93CF93DF93DC
:100BB000EC0181E0898B9C898D8998131CC0AC85E0
:100BC000BD8514968C91149785FF15C012966C9371
:100BD000AC85BD8580E414968C93EC85FD8585817C
:100BE0008F7D858381E090E0DF91CF911F910F9100
:100BF000FF90EF9008958091110180FF08C08091CF
:100C00001301888F8E898093130181E08F8BF62EDC
:100C10000C8910E00F5F1F4F0F731127E02E8D8995
:100C20008E1104C0CE010E94C305F9CFEC89EC0FF0
:100C3000FD2FF11DE75AFF4FF0820C8BEC85FD85EF
:100C400085818062CECFCF93DF93FC01218922235F
:100C5000C9F0EC018091110180FF08C0809113015F
:100C6000808F86898093130181E0878BEC85FD85D9
:100C7000858185FD03C0848186FD04C0CE010E946C
:100C8000C305F4CFDF91CF910895CF93DF9390E028
:100C9000FC01E056F04120812F3F89F0633071055F
:100CA00070F4FC01E654F041A08130E2A39FD00132
:100CB0001124BC5F6130710529F411962C93DF91EA
:100CC000CF9108958A5D9041EC01E881EF3F89F072
:100CD000CD014096E80FF92FF11D9FB7F8941296B9
:100CE0002C9380816230710539F4886080839FBFC6
:100CF000E6CFF0E0E0E0F1CF877FF8CF282F30E0BB
:100D0000F901E850F141E081EE2309F1E13021F0F1
:100D1000F0F0E63098F008954091010A2A5D3041E4
:100D2000F90120812C5F81E090E001C0880F2A95B5
:100D3000EAF7809584238093010A089580E1E89F73
:100D4000F0011124E05AF54F81818F7E818308954F
:100D5000FF920F931F93CF93DF93082F10E0F801BA
:100D6000E056F041F0809FEFF916A1F0EB018B32D5
:100D700010F40E947E06F801E654F041E08180E222
:100D8000E89FF0011124FC5F80818F2179F020978A
:100D900039F4F682DF91CF911F910F91FF90089562
:100DA000229711F4F782F6CFF582F4CFD801AA5D2D
:100DB000B0418C91309771F08F3F61F07096E80FE1
:100DC000F11D9FB7F8948081CD2B39F4877F808304
:100DD0009FBFE0CFF0E0E0E0F4CF8860F8CF0F9362
:100DE0001F93CF93082F10E0F801E056F041C08127
:100DF000CF3FB9F08B3210F40E947E06F801E65422
:100E0000F041E08180E2E89FF0011124FC5F8085E1
:100E1000C82381E090E009F480E0CF911F910F9109
:100E2000089580E090E0F9CF8B3210F40C94A8067E
:100E300008958B3210F40C9445060895CF92DF92FA
:100E4000EF92FF920F931F93CF93DF93EC016A0110
:100E50007B01022F8989882339F0E881F981028892
:100E6000F389E02DCE01099598898091E205892BBF
:100E70008093E2051FB7F89460E070E281EA97E0A2
:100E8000A70196010E94175169017A018FEFC81AD4
:100E9000D80AE80AF80AF694E794D794C794EC8540
:100EA000FD8586818D7F8683EC85FD8586818683A1
:100EB000198AA09123110A2E000CBB0BA7019601E1
:100EC0000E94DE5020E034E040E050E00E94B45048
:100ED000EC85FD85C20ED31EE41EF51EC086D186AC
:100EE000EC85FD850783EC85FD858681806C868396
:100EF000EC85FD858581806885838E8562E070E064
:100F00000E9419078F8561E070E00E9414078F85A9
:100F100061E070E00E9419071FBFDF91CF911F9120
:100F20000F91FF90EF90DF90CF900895E82FF0E0C1
:100F3000E051F1418E30B8F480818F30B0F480936D
:100F4000060681E08093080680910B0680FFFCCFA7
:100F50002FB7F89490911006809111062FBF892722
:100F60009827892708953E97E7CF8FEF90E008955F
:100F7000CF93DF938FB7F8942091E02A3091E12A44
:100F80004091E22A5091E32AE091BA0A9091B60A80
:100F900090FF06C02F5F3F4F4F4F5F4FE091BA0A5F
:100FA0008FBFA091DE2AB091DF2AC091DC2AD091B8
:100FB000DD2A0E94D350EC9F9001ED9F300D11244B
:100FC000620F731F811D911DDF91CF9108958F9244
:100FD0009F92AF92BF92CF92DF92EF92FF924B011E
:100FE0005C010E94B8076B017C01A8EEB3E0A5018B
:100FF00094010E94D350C60ED71EE81EF91EC616D5
:10100000D706E806F90618F40E94B807F8CF0E9440
:10101000B8076C157D058E059F05C8F3FF90EF900E
:10102000DF90CF90BF90AF909F908F9008952FB793
:10103000F8946091D82A7091D92A8091DA2A9091F7
:10104000DB2A2FBF08950F931F93CF93DF938C015B
:10105000EB0180915C2890915D28A0915E28B09171
:101060005F28892B8A2B8B2B51F40E9417086093E1
:101070005C2870935D2880935E2890935F280130F0
:10108000110539F0CF3FDC07A1F481E0809361289E
:1010900006C0CF3FDC0741F481E080936028DF91F8
:1010A000CF911F910F910895C0936528D093662822
:1010B000F6CFC0936328D0936428F1CF8F929F928C
:1010C000AF92BF92EF92FF921F93CF93DF93182FAF
:1010D000EB017A0189E00E9460049091C32D911187
:1010E00037C021E030E001C0220F1A95EAF78223D1
:1010F00011E009F410E00E94170811114FC0888018
:101100009980AA80BB8081149104A104B10411F5D7
:10111000688379838A839B838F819885029702975E
:1011200060F4112351F0F7018781908502970297AF
:1011300020F48185928587839087812FDF91CF91DD
:101140001F91FF90EF90BF90AF909F908F90089568
:101150001FEFD1CF1D81111167C0681979098A0964
:101160009B096D3271408105910590F081E08D837E
:101170008F8198858230910598F18430910508F02F
:1011800040C02D81222309F448C081E08E8339C0FC
:101190008C818111C1CF81E08C83BECF1C81112352
:1011A000B9F02D81211113C088809980AA80BB805D
:1011B000681979098A099B0989889A88092C000C81
:1011C000AA08BB0886169706A806B90688F210E09A
:1011D0001C821D821E82188219821A821B829CCF59
:1011E00089879A872D81222399F0019771F083E0F6
:1011F00090E08F8398870E9417086B877C878D8784
:101200009E871111E5CF11E087CF82E090E0F1CF0A
:10121000E1E08E278F839887F4CF29853A858987E7
:101220009A872F833887EDCF10E076CFAF92BF92A9
:10123000CF92DF92EF92FF920F931F93CF93DF93A2
:101240006C017B018B01040F151FEB015E01AE18D1
:10125000BF08C017D10759F06991D601ED91FC91F3
:101260000190F081E02DC6010995892B79F7C50120
:10127000DF91CF911F910F91FF90EF90DF90CF9072
:10128000BF90AF900895EF92FF920F931F93CF936B
:10129000DF93C82FD0E0A09695E0CC0FDD1F9A9584
:1012A000E1F7E984F82EFF0CFF0CFF0C01E010E0E1
:1012B0008E2D8023A9F02F2D210F30E0220F331F18
:1012C000F901E75BF44D80819181892B49F0019010
:1012D000F081E02D2751354DD9018D919C910995D3
:1012E0001F5F000F183021F7E986DF91CF911F9122
:1012F0000F91FF90EF900895FC01A485B58511969C
:101300008C91119781FD1BC06C9182898F5F8F73C7
:101310009389981739F0A289AE0FBF2FB11D599646
:101320006C93828BE756FF4F80819181009741F04B
:10133000DC01ED91FC910190F081E02D09948C91FC
:10134000089581E00895FC019085957081E09530C5
:1013500009F080E00895CF92DF92EF92FF920F9311
:101360001F93CF93DF93EC0188858B7F8887E8817B
:10137000F9810190F081E02DCE010995182F888523
:10138000869581701817B9F00E9417086A837B83CD
:101390008C839D83888592E089278887888582FB56
:1013A000882780F9DF91CF911F910F91FF90EF90E7
:1013B000DF90CF9008950E941708CA80DB80EC80F0
:1013C000FD80AB01BC014C195D096E097F098E815E
:1013D0009F81B0E0A0E0481759076A077B07F0F249
:1013E000888581701817D1F20E9417086A837B8361
:1013F0008C839D83888591E08927846088870E94FB
:10140000170809851A852B853C85601B710B820B9B
:10141000930B6D877E878F87988B0E94170869874B
:101420007A878B879C87BACFCF93DF93EC0118869E
:10143000E881F9810190F081E02D0995882319F068
:101440008885836088870E9417086A837B838C83E2
:101450009D83DF91CF910895862FBA010C941907CF
:10146000FC01818930E020E08B3218F40E94EF0605
:101470009C0181E0232B09F480E008950895EF9208
:10148000FF920F931F93CF93DF937C01EB018B01AE
:10149000040F151FC017D10759F0D701ED91FC912A
:1014A0000480F581E02D6881C70109958993F2CF09
:1014B000DF91CF911F910F91FF90EF9008950F93BF
:1014C0001F93CF93DF93EC018B018091C008E881DB
:1014D000F9810480F581E02D86FD13C0612FCE01D6
:1014E0000995182FE881F9810480F581E02D602F9E
:1014F000CE010995082FC801DF91CF911F910F915F
:101500000895CE010995082FE881F9810480F581BD
:10151000E02D612FCE010995182FEDCF00006093CB
:10152000C4088091C30887FFFCCF8091C408089548
:101530008F929F92AF92BF92CF92DF92EF92FF92E3
:101540000F931F93CF93DF93FC018085882319F0BD
:1015500081FF0EC07894DF91CF911F910F91FF9082
:10156000EF90DF90CF90BF90AF909F908F900895B5
:1015700080FFF1CF82849384A484B584C12CD12CC4
:10158000760110E09401A501B601C701A0E00E9418
:10159000DB5599F1217030E040E050E060E070E010
:1015A00080E090E00E94DB55D9F0D0E0C0E010333D
:1015B00070F4C12FC695C695C69580E2C89FE0011C
:1015C0001124C05FDB4F812F8770C80FD11DCF0161
:1015D000810F911DDC0152968C919881892B888313
:1015E0009401A501B601C70101E00E94C05549015F
:1015F0005A016B017C011F5FC5CF86849784A08848
:10160000B188C12CD12C760110E29401A501B6015C
:10161000C701A0E00E94DB5509F49DCF217030E0A6
:1016200040E050E060E070E080E090E00E94DB5538
:10163000D9F0D0E0C0E0103370F4C12FC695C69544
:10164000C695B0E2CB9FE0011124C05FDB4F812F34
:101650008770C80FD11DCF01810F911DDC015296FB
:101660008C919881892B88839401A501B601C701CB
:1016700001E00E94C05549015A016B017C011F5FC6
:10168000C4CFFC016F3F710581F1808581FD2DC0C4
:10169000603271055CF581E090E002C0880F991F0F
:1016A0006A95E2F780959095092E000CAA0BBB0B6A
:1016B000428553856485758584239523A623B723A6
:1016C00082879387A487B58782859385A485B5850E
:1016D000892B8A2B8B2B49F486859785A089B18924
:1016E000892B8A2B8B2B09F410860895605271097F
:1016F00081E090E002C0880F991F6A95E2F780951B
:101700009095092E000CAA0BBB0B46855785608966
:10171000718984239523A623B72386879787A08B77
:10172000B18BD2CFFC016F3F7105E9F160337105D8
:101730001CF082E080870895808581608087603218
:101740007105C4F481E090E002C0880F991F6A958A
:10175000E2F7092E000CAA0BBB0B4285538564856A
:101760007585842B952BA62BB72B82879387A4870F
:10177000B58708956052710981E090E002C0880F3A
:10178000991F6A95E2F7092E000CAA0BBB0B468540
:10179000578560897189842B952BA62BB72B86875B
:1017A0009787A08BB18B0895E0ECF8E020812E7F25
:1017B0002083FC0117820895E0ECF8E082818E7F9F
:1017C00082830895E0ECF8E082818160828308954D
:1017D0000F9391E09093422A1092412A60933F2AFE
:1017E0007093402A40933E2A20933D2A10923C2A2F
:1017F00010923B2A00933A2A880F8093392A23E0DB
:1018000030E044E050E080913E2A882341F020936C
:10181000372A3093382A8091392A8E7F0BC08091E5
:101820003D2A882351F04093372A5093382A8091DB
:10183000392A81608093A70808C080913E2A8111CF
:1018400004C080913D2A882311F38091412A882386
:10185000E1F38091412A8330B1F280913D2A8823BF
:1018600021F080913B2A0F9108958091412A823086
:1018700031F0853031F0813031F480E0F4CF81E017
:10188000F2CF83E0F0CF84E0EECFE0EAF8E091859C
:101890009066918722E030E02093372A3093382AEF
:1018A0008093292A1092282A089581E08093282A7B
:1018B0001092292A93E09093AA089091AB0891FF87
:1018C00010C01092352AE091262AF091272A099516
:1018D0008093342A85E090E08093372A9093382AC9
:1018E00008951092362A8093332A86E090E0F4CF50
:1018F0008F929F92AF92BF92CF92DF92EF92FF9220
:10190000CF93DF9360342DE0720723E082079105C7
:1019100008F454C0611525E372072CE08207910595
:1019200008F445C060387F448241910508F046C004
:10193000C8E7D0E020E432E44FE050E08090112886
:1019400090901228A0901328B0901428C501B401DB
:101950000E94175169017A018AE0C81AD108E1088A
:10196000F108C501B40120E432E44FE050E00E94E8
:101970001751DE010E94D35028EE33E040E050E0E2
:101980000E941751C21AD30AE40AF50AF694E794A2
:10199000D794C794C092A608DF91CF91FF90EF90A3
:1019A000DF90CF90BF90AF909F908F900895CCE242
:1019B000D1E020E83AE146E050E0C0CFC8EED3E005
:1019C00020EA36E841E050E0B9CF6093242A7093D2
:1019D000252A08956093222A7093232A0895E0917E
:1019E000242AF091252A309741F01092212A109252
:1019F000202A09958091202A089580E00895E09199
:101A0000222AF091232A309759F030911F2A2091F1
:101A10001E2A321728F010921F2A80931E2A09943A
:101A200008950895E0911F2A80911E2AE81730F446
:101A3000F0E0E256F64D808190E008958FEF9FEF41
:101A4000089590911F2A80911E2A2FEF3FEF98173B
:101A500048F4E92FF0E0E256F64D208130E09F5F38
:101A600090931F2AC901089580911E2A90911F2AE0
:101A7000891B990B0895CF92DF92EF92FF920F93FB
:101A80001F93CF93DF937C018A01EB016B01C40E9E
:101A9000D51ECC15DD0551F06991D701ED91FC9172
:101AA0000190F081E02DC7010995F3CFC801DF91C6
:101AB000CF911F910F91FF90EF90DF90CF900895FD
:101AC0002091202A27FF08C021E030E0FC0122837A
:101AD000338390E080E008958091212AE82FF0E0A0
:101AE000E25EF64D60838F5F8093212A8093202AE7
:101AF00081E090E00895DC01ED91FC91008CF18D86
:101B0000E02D61E009940F938091372A9091382A53
:101B10000197A1F48091422A811112C0062F20E082
:101B20004091202A6EE179E280911D290E94E80B04
:101B30001092212A1092202A0F91089580E0F8CF68
:101B400081E0F6CF60931D291092212A1092202A5D
:101B50000895DC01ED91FC91048CF58DE02D21E0E0
:101B600009940F938EE999E280932A2A90932B2A65
:101B70008091372A9091382A0197C9F48091422A9E
:101B8000811117C0FA014138510510F0E0E8F0E08A
:101B9000022F862F2E2F40E070E060E00E94E80BBD
:101BA00010921F2A80931E2A90E00F91089580E0E2
:101BB000F7CF81E0F5CFCB01BA010C94780CE0EAC5
:101BC000F8E01382168281E08583148611861092D4
:101BD000372A1092382A089510921F2A10921E2A2E
:101BE0001092212A1092202A8091372A9091382A27
:101BF000892BD9F482E090E08093372A9093382A99
:101C00001092362A1092352A1092282A1092292AE8
:101C100010921C291092332A660F6093AC0881EE53
:101C20008093A90881E08093A3088FEE9CE08093C5
:101C3000262A9093272A8EE199E280932C2A90936A
:101C40002D2A8FEF9CE08093312A9093322A8EE9DF
:101C500099E280932E2A90932F2A80E88093302A4D
:101C6000089510921F2A10921E2A1092212A109273
:101C7000202A8091372A9091382A892B41F562E0F9
:101C800070E086E10E94450662E070E087E10E9414
:101C900045068091E3058093E30581E090E0809321
:101CA000372A9093382A10923B2A10923C2A10929D
:101CB000422A1092412A81EC8093A30860EA76E8D8
:101CC00081E090E00E94780C81E08093A50808955F
:101CD000FC01A5A1B6A18C9192A589238C93A5A105
:101CE000B6A18C9191A5892B8C930895DC019396D4
:101CF000ED91FC919497908198968C9189238083A3
:101D00000895DC019396ED91FC91949790819796BC
:101D10008C91892B80830895DC019196ED91FC9143
:101D20009297908196968C91892380830895DC0107
:101D30009196ED91FC919297908195968C91892B3B
:101D400080830895CF92DF92EF92FF921F93CF93FB
:101D5000DF93EC016A017B018DA981112BC08F2DCE
:101D60009927AA27BB278093C4088091C30887FFBF
:101D7000FCCFC701AA27BB278093C4088091C30862
:101D800087FFFCCFBB27AF2D9E2D8D2D8093C408E0
:101D90008091C30887FFFCCFC092C4088091C3081C
:101DA00087FFFCCFDF91CF911F91FF90EF90DF90E5
:101DB000CF9008958130B1F410E2CE01F7FE0FC04C
:101DC0000E94970ECE010E94810ECE010E94760ED7
:101DD000CC0CDD1CEE1CFF1C115079F7E3CF0E94E8
:101DE0008C0EF0CFEF8DF8A18F2D9927AA27BB2756
:101DF0008083CE010E94680EEF8DF8A1C701AA274B
:101E0000BB278083CE010E94680EEF8DF8A1BB270F
:101E1000AF2D9E2D8D2D8083CE010E94680EEF8DFB
:101E2000F8A1C082CE01DF91CF911F91FF90EF907A
:101E3000DF90CF900C94680EFF920F931F93CF9377
:101E4000DF93EC018B018DA9811112C01093C4089E
:101E50008091C30887FFFCCF0093C4088091C3081A
:101E600087FFFCCFDF91CF911F910F91FF900895D5
:101E70008130B1F490E1F92ECE0117FF0EC00E941F
:101E8000970ECE010E94810ECE010E94760E000FA9
:101E9000111FFA94F110F0CFE5CF0E948C0EF1CF14
:101EA000EF8DF8A11083CE010E94680EEF8DF8A18E
:101EB0000083CE01DF91CF911F910F91FF900C9481
:101EC000680E0F931F93CF93DF93EC01162F8DA90C
:101ED00081110BC06093C4088091C30887FFFCCFB9
:101EE000DF91CF911F910F910895813099F408E00F
:101EF000CE0117FF0CC00E94970ECE010E94810EEA
:101F0000110FCE010E94760E015091F7E9CF0E9489
:101F10008C0EF3CFEF8DF8A16083CE01DF91CF91CE
:101F20001F910F910C94680ECF93DF93EC01ED8D10
:101F3000FE8D80819CA989238083CE010E94610F40
:101F4000ED8DFE8D80819BA9892B8083DF91CF91C0
:101F500008958F929F92AF92BF92CF92DF92EF92AD
:101F6000FF920F931F93CF93DF93EC0189AD9AAD4E
:101F7000680F791F8BAD9CAD480F591F2150310957
:101F8000260F371F4901B12CA12CCB01B0E0A0E0F6
:101F9000DC0199278827882A992AAA2ABB2A68015E
:101FA00081E0C81AD108C40ED51EF12CE12C70E0D6
:101FB00060E0BA0155274427C42AD52AE62AF72A21
:101FC0006AE2CE010E94940FB501A401CE010E94E5
:101FD000A20E6BE2CE010E94940FB701A601CE01C2
:101FE0000E94A20E6CE2CE01DF91CF911F910F9162
:101FF000FF90EF90DF90CF90BF90AF909F908F9029
:102000000C94940FDC01D5962C91D59721110AC020
:102010005F968D919C91DC01ED91FC910088F18996
:10202000E02D099408950F931F93CF93DF93EC0154
:102030002DA9211121C0DC018F8D98A1EC01E8812F
:10204000F9810684F785E02D91960C9191979296EF
:102050001C91929793962C91939794963C91949778
:1020600095964C91959796965C91969797966C91CC
:10207000979798967C910995DF91CF911F910F9139
:1020800008950F931F93CF93DF93EC018B010E9470
:1020900013108FA987FD06C0EB8DFC8D80819AA956
:1020A00089238083ED8DFE8D80819CA98923808387
:1020B00066E3CE010E94610FED8DFE8D80819BA9AC
:1020C000892B80838DA9F8018230A1F06081CE0137
:1020D0000E94610F8FA987FD06C0EB8DFC8D80816A
:1020E00099A9892B8083CE01DF91CF911F910F9108
:1020F0000C94021088A9882349F360817181CE0174
:102100000E941C0FE7CFCF93DF931F92CDB7DEB7AE
:10211000FC0119826370668BDC01AD5BBF4F2C91B3
:1021200030E011968C9190E0623031F06330C9F06C
:10213000613081F040EC498321AF32AF83AF94AF7F
:10214000BE016F5F7F4FCF010E9441100F90DF9162
:10215000CF91089540EA498323AF34AF81AF92AF66
:10216000EFCF40E6F8CF0F931F93CF93DF931F92EB
:10217000CDB7DEB7FC0119826370668BDC01A85B0A
:10218000BF4F2D913C91119712968D919C91623089
:10219000D1F1633009F440C08F010C5B1F4F6130F7
:1021A000F9F040EC4983AF014D5B5F4FDA014C9190
:1021B00050E041AF52AFD8014C9150E043AF54AF23
:1021C0002087318782879387BE016F5F7F4FCF0162
:1021D0000E9441100F90DF91CF911F910F910895B0
:1021E00040EA4983D8014C9150E041AF52AFDF0142
:1021F000AA5BBF4F4C9150E043AF54AF2287338767
:1022000080879187E1CFDF01AA5BBF4F4C9150E0FF
:1022100041AF52AF1196D0CF40E64983DF01A95BB1
:10222000BF4F4C9150E041AF52AF1497E3CF1F9393
:10223000CF93DF93EC01162FE881F9810284F385B7
:10224000E02D0995112371F06DADCE010E94940F20
:10225000E881F9810688F789E02DCE01DF91CF91E1
:102260001F9109946EADF1CFAF92BF92CF92DF92E2
:10227000EF92FF920F931F93CF93DF93EC0177FDC3
:1022800038C088859985681779079CF557FD31C056
:102290008A859B854817590764F569017A015B01B6
:1022A000E881F9810284F385E02DCE010995E8816A
:1022B000F98102A4F3A5E02D01E010E021E030E077
:1022C000A701B501CE010995B601CE010E941C0FF0
:1022D000E881F9810688F789E02DCE01DF91CF9161
:1022E0001F910F91FF90EF90DF90CF90BF90AF9034
:1022F0000994DF91CF911F910F91FF90EF90DF90A4
:10230000CF90BF90AF9008958F929F92AF92BF925F
:10231000CF92DF92EF92FF920F931F93CF93DF93B1
:10232000EC0149015701E881F98102A4F3A5E02DF0
:1023300009959401D8010E94AF556B017C01C1142D
:10234000D104E104F10409F481C08DA9811119C0FF
:1023500081E0C81AD108E108F1088FEFC816D80645
:10236000E806F80609F472C0B092C4088091C30868
:1023700087FFFCCFA092C4088091C30887FFFCCFE1
:10238000E7CF813099F581E0C81AD108E108F1085A
:102390008FEFC816D806E806F80609F457C00B2DCB
:1023A00018E0CE0107FF1CC00E94970ECE010E94CC
:1023B000810ECE010E94760E000F115091F70A2D6A
:1023C00018E0CE0107FF0FC00E94970ECE010E94B9
:1023D000810ECE010E94760E000F115091F7D3CFDF
:1023E0000E948C0EE3CF0E948C0EF0CFBA1016C064
:1023F000CC0CDD1CEE1CFF1CEF8DF8A1B08281E03F
:10240000C81AD108E108F1088FEFC816D806E80607
:10241000F806E1F0CE010E94680EF1CF81E0C81A03
:10242000D108E108F1088FEFC816D806E806F806CB
:1024300069F0EF8DF8A1B082CE010E94680EEF8D99
:10244000F8A1A082CE010E94680EE8CFDF91CF9163
:102450001F910F91FF90EF90DF90CF90BF90AF90C2
:102460009F908F9008958F929F92AF92BF92CF923C
:10247000DF92EF92FF920F931F93CF93DF934C0164
:10248000EB016A01590137FF07C0C9010196C80F66
:10249000D91FB194A194B108F401A085B185CA17E0
:1024A000DB070CF058C017FF07C0C8010196C80E23
:1024B000D91E119501951109F40182859385C816DD
:1024C000D9060CF048C0FE01EA0DFB1DAF014150DA
:1024D000510957FD40C0B601600F711F9B0121508B
:1024E000310937FD38C0D7FF03C05F01D0E0C0E03D
:1024F000D7FE03C08B01D12CC12C4A175B071CF0FF
:102500005D01AC1ABD0A281739071CF08C010C19A3
:102510001D09D401ED91FC910284F385E02DC401E5
:1025200009959501A601BE01C4010E948411D40140
:10253000ED91FC910688F789E02DC401DF91CF91E0
:102540001F910F91FF90EF90DF90CF90BF90AF90D1
:102550009F908F900994DF91CF911F910F91FF90E1
:10256000EF90DF90CF90BF90AF909F908F900895A5
:10257000EF92FF920F931F932115310529F001155A
:10258000110511F00E9433121F910F91FF90EF90EF
:1025900008958F929F92AF92BF92CF92DF92EF9267
:1025A000FF920F931F93CF93DF935C014B016A015E
:1025B000E90177FD52C0DC0118968D919C91681756
:1025C00079070CF04AC0209709F447C037FF07C0CD
:1025D000C9010196C80ED91ED195C195D109F50141
:1025E00082859385C816D906C4F5A6014C0F5D1FD8
:1025F0009A012150310937FD30C0D7FE03C0EA01EE
:10260000D12CC12C281739071CF0EC01CC19DD099D
:10261000D501ED91FC910284F385E02DC50109956A
:1026200078018E0121E030E0A601B401C5010E94CD
:102630008411D501ED91FC910688F789E02DC50143
:10264000DF91CF911F910F91FF90EF90DF90CF908E
:10265000BF90AF909F908F900994DF91CF911F9181
:102660000F91FF90EF90DF90CF90BF90AF909F9031
:102670008F9008958F929F92AF92BF92CF92DF92E8
:10268000EF92FF920F931F93CF93DF935C016B0147
:102690004A01E90157FD52C0DC011A968D919C91C7
:1026A000481759070CF04AC0209709F447C037FF74
:1026B00007C0C9010196C80ED91ED195C195D1098F
:1026C000F50180859185C816D906C4F5A6014C0F81
:1026D0005D1F9A012150310937FD30C0D7FE03C07C
:1026E000EA01D12CC12C281739071CF0EC01CC19B8
:1026F000DD09D501ED91FC910284F385E02DC50142
:102700000995780101E010E09E01A401B601C50120
:102710000E948411D501ED91FC910688F789E02D86
:10272000C501DF91CF911F910F91FF90EF90DF9046
:10273000CF90BF90AF909F908F900994DF91CF91F1
:102740001F910F91FF90EF90DF90CF90BF90AF90CF
:102750009F908F900895EF92FF920F931F93CF93C6
:10276000DF9377FD32C0DC011896ED91FC916E1776
:102770007F075CF52115310541F137FF07C0F901ED
:1027800031964E0F5F1F319521953109DC011A9664
:10279000ED91FC914E175F07C4F4EA01C20FD31FFD
:1027A000DE011197B7FD11C057FF03C09E0150E035
:1027B00040E0AE17BF071CF09F01241B350B7801CA
:1027C000890121E030E00E948411DF91CF911F91B7
:1027D0000F91FF90EF900895EF92FF920F931F9348
:1027E000CF93DF9357FD31C0DC011A96ED91FC9138
:1027F0004E175F0754F52115310539F137FF07C032
:10280000F90131966E0F7F1F319521953109DC0159
:102810001896ED91FC916E177F07BCF4EB01C20F87
:10282000D31FDE011197B7FD10C077FF03C09E01D3
:1028300070E060E0AE17BF071CF09F01261B370B4E
:10284000780101E010E00E948411DF91CF911F9187
:102850000F91FF90EF9008958F929F92AF92BF9249
:10286000CF92DF92EF92FF920F931F93CF93DF935C
:1028700047012115310509F44BC00115110509F473
:1028800047C037FF07C0F90131966E0F7F1F3195A2
:1028900021953109DC011896AD90BC906A157B0535
:1028A000BCF517FF07C0F80131964E0F5F1F119559
:1028B00001951109DC011A96ED91FC914E175F0705
:1028C0003CF56B01C20ED31EE6012197D7FD20C057
:1028D0007A01E00EF11ED7011197B7FD19C077FFFD
:1028E00003C0960170E060E057FF03C0870150E02D
:1028F00040E0CA15DB051CF09501261B370BAE170F
:10290000BF071CF08F01041B150B74010E9484117A
:10291000DF91CF911F910F91FF90EF90DF90CF90BB
:10292000BF90AF909F908F900895EF92FF920F937A
:102930001F93CF93DF93EC0177FD22C088859985A3
:1029400068177907ECF457FD1BC08A859B854817EB
:102950005907B4F47901E881F98102A4F3A5E02DC7
:1029600001E010E021E030E0CE010995B701CE0191
:10297000DF91CF911F910F91FF90EF900C941C0F5E
:10298000DF91CF911F910F91FF90EF900895DC019F
:10299000D7962C91D79727FD09C05B96ED91FC91B6
:1029A0005C972081D1963C91232B20830C940210BC
:1029B000CF93DF93EC010E9413108FA987FD06C00F
:1029C000EB8DFC8D80819AA989238083DF91CF9143
:1029D00008950895FC016370668B8481958126813A
:1029E0003781613039F0633029F080879187228701
:1029F00033870895208731878287938708952F92A0
:102A00003F924F925F926F927F928F929F92AF927E
:102A1000BF92CF92DF92EF92FF920F931F93CF93CB
:102A2000DF93CDB7DEB76A97CDBFDEBF898F9A8FB0
:102A300069837A834A01D22E0F8318873701BC2C11
:102A4000DC0159962D913C915A972115310509F0D9
:102A500012C118968D919C911997681779070CF0FF
:102A6000D4C11A968D919C91481759070CF0CDC18D
:102A70004C2C512CB6E0CB9E600D711D11246B8740
:102A80007C87161617060CF0C0C1EA2DF0E0E98726
:102A9000FA8793E0EE0FFF1F9A95E1F7EF87F88B27
:102AA000CF01840F951F181619060CF0AEC1A98D21
:102AB000BA8D58968C91811104C0BFEABD1508F4F7
:102AC000D394A98DBA8DED91FC9111970284F38571
:102AD000E02DCD010995B5E0DB9EC0011124E9810F
:102AE000FA81EB83FC83312C212C9C0128513D4F32
:102AF0002F8B388F4A2D50E04D8B5E8BEF89F88DF0
:102B0000E20DF31D44918D829E82D12CC12C6981EE
:102B10007A81620D731D698B7A8B842F90E08B8B89
:102B20009C8BE98DFA8DA081B18140FF7FC0F1E0DF
:102B3000BF126CC0AF126AC01C96ED91FC912F8140
:102B40003885A4014C0D5D1D69897A89898D9A8D1E
:102B50000995EB89FC89F595E7954E2F5FEFC51A2E
:102B6000D50A6D817E818D899E89680F791F6D835D
:102B70007E8398E0C916D10481F6AFEF2A1A3A0A8B
:102B8000EB81FC81E40DF51DEB83FC83F5E02F1652
:102B9000310409F0B3CF2F81388526153705B9F0F8
:102BA000A98DBA8DED91FC91B1E0BB1254C0AB126E
:102BB00052C069817A816B5F7F4F0088F189E02D77
:102BC000830128E030E0A401898D9A8D0995A98DB3
:102BD000BA8DED91FC9111970688F789E02DCD0112
:102BE0006A96CDBFDEBFDF91CF911F910F91FF900D
:102BF000EF90DF90CF90BF90AF909F908F907F909D
:102C00006F905F904F903F902F9009941E96ED919A
:102C1000FC91EF80F88409851A8592014D815E81CF
:102C20006B817C81898D9A8D099593CF2F81388511
:102C30002615370509F48DCF31E0B31207C0A31272
:102C400005C01C96ED91FC9193017BCF1E96ED91F2
:102C5000FC917301E0CF6B857C856419750906844E
:102C6000F785E02D73010F8518899201A401898DE4
:102C70009A8D0995ACCFF90134969491329745918C
:102C80005491D91AB7E0DB9E400D511D1124F90172
:102C9000259134912B8B3C8BFA0125903490FA01CD
:102CA0003296749031963491398B32966490319685
:102CB000449041E04C1518F04A1508F07FC0662D8D
:102CC000062C000C770B6B837C83842D042C000C6A
:102CD000990B8D839E83A98DBA8DED91FC911197EF
:102CE0000284F385E02DCD010995512CD12CC12C06
:102CF000EA2DF0E0E987FA872B2D30E02B873C871F
:102D0000A401440D511D47FC5A954F8B588F698182
:102D10007A81660D711D67FC7A956D877E8779894A
:102D2000C71608F054CF2C2D30E04D815E81420F44
:102D3000531FA985BA854A9FC0014B9F900D5A9F8A
:102D4000900D1124FC01E80DF91DEF87F88B852DFE
:102D5000612C4F89588D420F531F4D8B5E8B67142A
:102D600008F050C044244394480E877041F4C101D8
:102D70000196EB89FC89E20DF31DD4901C01D7FE6E
:102D800019C0A98DBA8DED91FC91662D70E0B1E06E
:102D9000BB1219C0AB1217C02D853E85620F731F81
:102DA0000484F585E02D2F8138854D895E89898DD4
:102DB0009A8D0995DD0C6394842DD1CF1D821E82DE
:102DC0001B821C8288CF4B815C81640F751FAB8591
:102DD000BC856A9FC0016B9F900D7A9F900D112456
:102DE00069817A81680F791F0684F785E02DEF806D
:102DF000F88409851A859D014F855889898D9A8D9A
:102E00000995D8CF570CC3948ACF6A96CDBFDEBF41
:102E1000DF91CF911F910F91FF90EF90DF90CF90B6
:102E2000BF90AF909F908F907F906F905F904F90EA
:102E30003F902F9008958F929F92AF92CF92EF92F2
:102E4000FF920F931F93CF93DF93EC01262F898D71
:102E50009A8D009709F051C06A30D1F41C861D8606
:102E60008D8948E0849F900111248E859F85820F73
:102E7000931F8E879F8781E090E0DF91CF911F9114
:102E80000F91FF90EF90CF90AF909F908F9008950B
:102E90006D3089F3CC88AD888F898823C1F08C850B
:102EA0009D8536E0C39E800D911D1124488559856E
:102EB0004817590764F44E855F851C861D8638E0E7
:102EC000A39EC0011124840F951F8E879F87EA88D7
:102ED000FB88088919894E855F856C857D85CE01C3
:102EE0000E94FF142C898C859D8546E0249F800DCF
:102EF000911D11248C879D87BECF6A3069F41C8692
:102F00001D86FC013896E4912D898E859F85E29F70
:102F1000800D911D1124ADCF6D3009F4ACCFFC01B3
:102F200034963491631708F4A6CF3296E491E617ED
:102F300008F4A1CFFC01329685909490462F431B54
:102F4000342F47E0349F800C911C1124F4013296F9
:102F500034913196E4913323A9F1EE2399F1CC8891
:102F6000F4013596E491AD884F89442301F10E2E8A
:102F7000000CFF0BE30FF11DCE9EA001CF9E500D64
:102F800011246C857D85460F571F688579856417E8
:102F900075076CF44E855F851C861D86FC0138968E
:102FA000E491AE9E400D511D11244E875F87EA8843
:102FB000FB88088919894E855F856C857D85CE01E2
:102FC0000E94FF14F4013496E4912C898C859D8530
:102FD000E29F800D911D11248DCF6F927F928F9271
:102FE0009F92AF92BF92CF92DF92EF92FF920F9398
:102FF0001F93CF93DF93EC016B015A013901480114
:10300000E881F9810284F385E02D0995E881F98151
:103010000288F389E02D87019301A501B601CE0155
:103020000995A501480D591D41505109E881F981C3
:103030000288F389E02D9301B601CE010995E8815C
:10304000F9810088F189E02D9401A501B601CE0136
:103050000995C60CD71CB60161507109E881F98148
:103060000088F189E02D9401A501CE010995E88140
:10307000F9810688F789E02DCE01DF91CF911F916C
:103080000F91FF90EF90DF90CF90BF90AF909F9007
:103090008F907F906F9009946F927F928F929F9202
:1030A000AF92BF92CF92DF92EF92FF920F931F9356
:1030B000CF93DF935C01EB016A014901380187017D
:1030C000DC01ED91FC916217730719F56416750622
:1030D0002CF0962D872D3A01C92ED82E960126194F
:1030E00037092F5F3F4F048CF58DE02DA301BE0102
:1030F000C5010995DF91CF911F910F91FF90EF903E
:10310000DF90CF90BF90AF909F908F907F906F9007
:1031100008954615570591F42617370724F0892D91
:103120004B01C22FD82F9E01281939092F5F3F4F1D
:10313000068CF78DE02DA601B401DACF0284F38569
:10314000E02D0995D501ED91FC910488F589E02DDC
:1031500083019401A601BE01C5010995D501ED9138
:10316000FC910688F789E02DC501DF91CF911F9171
:103170000F91FF90EF90DF90CF90BF90AF909F9016
:103180008F907F906F900994EF92FF920F931F930F
:10319000DC011A960D911C911B9718962D913C916C
:1031A0001997ED91FC9100A0F1A1E02D7B0150E079
:1031B00040E070E060E009951F910F91FF90EF9063
:1031C00008954F925F926F927F928F929F92AF92EB
:1031D000BF92CF92DF92EF92FF920F931F93CF9304
:1031E000DF936C012B015A0139014801DC01ED919B
:1031F000FC910284F385E02D0995E201640C751CB5
:10320000D601ED91FC91C615D7055CF40088F189D3
:10321000E02D87019401A501BE01C6010995219603
:10322000EFCF0688F789E02DC601DF91CF911F917E
:103230000F91FF90EF90DF90CF90BF90AF909F9055
:103240008F907F906F905F904F9009948F929F9294
:10325000AF92BF92CF92DF92EF92FF920F931F93A4
:10326000CF93DF93EC015B014A016901E881F981A9
:103270000284F385E02D099595012C0D3D1D21500B
:103280003109E881F9810488F589E02D780184010C
:10329000A401B501CE010995E881F9810688F78975
:1032A000E02DCE01DF91CF911F910F91FF90EF9014
:1032B000DF90CF90BF90AF909F908F9009948F92A6
:1032C0009F92AF92BF92CF92DF92EF92FF920F93B5
:1032D0001F93CF93DF93EC015B014A0169017801F1
:1032E000E881F9810284F385E02D0995C80CD91C89
:1032F000860101501109E881F9810488F589E02DE2
:103300009501A401B501CE010995E881F9810688EE
:10331000F789E02DCE01DF91CF911F910F91FF90A2
:10332000EF90DF90CF90BF90AF909F908F900994D7
:10333000EF92FF920F931F93DC01ED91FC9100A09F
:10334000F1A1E02D09951F910F91FF90EF90089545
:103350000F931F93DC01ED91FC91068CF78DE02D0E
:1033600009951F910F9108950F931F93DC01ED9123
:10337000FC91048CF58DE02D09951F910F91089516
:10338000DC01ED91FC910084F185E02D09942F92F0
:103390003F924F925F926F927F928F929F92AF92E5
:1033A000BF92CF92DF92EF92FF920F931F93CF9332
:1033B000DF93CDB7DEB72697CDBFDEBF3C016A01F4
:1033C0002D833E83EB82FC825801A41AB50AB7FE16
:1033D00003C0B194A194B1088D809E80861A970A8B
:1033E00097FE03C09194819491088A149B045CF029
:1033F000902F812F0D811E819D838E839C2D8D2D7D
:103400006B01692F782F0C151D055CF09D818E8155
:103410006D837E83692F782F902F812F8601C92E8F
:10342000D82E1601201A310A2B012D813E81421A15
:10343000530A57FE03C0519441945108710137FE5D
:1034400003C03FEFE31AF30AF594E7948D819E8160
:10345000861797075CF5A1E0B0E0A983BA83C01690
:10346000D1064CF1D301ED91FC910484F585E02D5A
:103470002B813C81A8016D817E818A149B041CF004
:103480004D815E81B801C3010995E418F508F7FE86
:103490000AC02D813E8189819A81280F391F2D8391
:1034A0003E83E20CF31C0F5F1F4FD9CF2FEF3FEF8E
:1034B00029833A83D4CF2696CDBFDEBFDF91CF914B
:1034C0001F910F91FF90EF90DF90CF90BF90AF9042
:1034D0009F908F907F906F905F904F903F902F9034
:1034E0000895089590E080E00895DC01ED91FC914D
:1034F0000088F189E02D23E030E00994CF92DF923B
:10350000EF92FF920F931F93CF93DF93FC012781DC
:103510003085225031092230310530F58C010E946E
:103520001708F801C785D089038514852585368558
:10353000601B710B820B930B9E010D2E000C440B34
:10354000550B0E941751AE01D7FF02C04F5F5F4F6E
:10355000559547956A01550FEE08FF0821E0C616FC
:10356000D706E806F90608F020E0822FDF91CF9118
:103570001F910F91FF90EF90DF90CF900895862FCD
:1035800090919F2A9923A1F06CE00E948955E92F20
:10359000F0E0EE0FFF1FE857F1418081918197FD28
:1035A00007C0809335289093362881E08093A12A24
:1035B0000895FC012081318142815381FB016081AA
:1035C0007181828193810E9448510E942C52CB01CB
:1035D0000895CF92DF92EF92FF920F931F93CF93B4
:1035E000DF936C019A018BE1869FE001879FD00DEC
:1035F0001124F12CE12C0BE110E0AE01B60184ECBA
:103600009DE20E94B812E4ECFDE2C486D5862396C2
:10361000C687D787DF91CF911F910F91FF90EF90D1
:10362000DF90CF90089510920D2910920E291092DC
:103630000F29109210291092BD2A1092BE2A1092C2
:1036400038281092392810923A2810923B2810926C
:10365000092910920A291092072910920829089521
:103660004F925F926F927F928F929F92AF92BF9292
:10367000CF92DF92EF92FF920F931F93CF93DF933E
:10368000CDB7DEB72E97CDBFDEBF80914528909194
:103690004628029709F04FC12091D12A298381E061
:1036A00082278093C02A0E94B8074B015C013981B0
:1036B000332309F438C18091A2289091A328A091C6
:1036C000A428B091A528A5019401281B390B4A0B09
:1036D0005B0BCA01B9010E94625269837A838B83B2
:1036E0009C83209131283091322840913328509189
:1036F00034280E94715320E030E044EB52E40E94F1
:10370000BA5120E030E040E05FE30E9449510E945E
:103710002C526B01770FEE08FF080091442C10919A
:10372000452CD8018C918E7F8C938C918670823041
:1037300009F45FC0843051F081110FC044E0CC0C1B
:10374000DD1CEE1CFF1C4A95D1F707C062E0F69421
:10375000E794D794C7946A95D1F780E090E0A1E010
:10376000B0E08093522C9093532CA093542CB093A0
:10377000552C9701442755272B873C874D875E871B
:103780002093462C3093472C4093482C5093492C3F
:10379000C701B6018827992760934A2C70934B2C58
:1037A00080934C2C90934D2C232B242B252B09F408
:1037B00044C0412C512C32016394A3019201215049
:1037C0003109410951092D833E834F835887613068
:1037D000710581059105A9F4C701B6010E94175131
:1037E0002B873C874D875E874D805E806F80788415
:1037F000E4CF53E0CC0CDD1CEE1CFF1C5A95D1F736
:10380000ACCF60934A2C70934B2C80934C2C9093AC
:103810004D2C4092522C5092532C6092542C70920A
:10382000552C2B853C854D855E852093462C309309
:10383000472C4093482C5093492C8091522C9091C6
:10384000532CA091542CB091552C0197A109B1098A
:103850008093522C9093532CA093542CB093552CBE
:1038600040914A2C50914B2C60914C2C70914D2CD6
:10387000411551056105710561F04150510961091A
:10388000710940934A2C50934B2C60934C2C7093AD
:103890004D2C4091462C5091472C6091482C7091B2
:1038A000492C40934E2C50934F2C6093502C709386
:1038B000512C452B462B472B21F480914A2C90917B
:1038C0004B2CD8011C968D939C931D971A961D9294
:1038D0001C921B978C9181608C93C501B4010E944E
:1038E00062526B017C0120E030E040EC5FE36981D3
:1038F0007A818B819C810E9471539B01AC01C7012D
:10390000B6010E94495120E030E04AE754E40E94A9
:10391000BA510E9433526093CD2A7093CE2A80937D
:10392000CF2A9093D02A8092A2289092A328A09286
:10393000A428B092A5282E96CDBFDEBFDF91CF91EF
:103940001F910F91FF90EF90DF90CF90BF90AF90BD
:103950009F908F907F906F905F904F90089580918F
:10396000452890914628892B29F08091D12A8823D7
:1039700009F454C08091462A9091472AA091482A80
:10398000B091492A0196A11DB11D8093462A9093BA
:10399000472AA093482AB093492A809116289091EB
:1039A00017284091462A5091472A6091482A7091E1
:1039B000492A092E000CAA0BBB0B481759076A07A6
:1039C0007B0748F081E090E08093C32A9093C42A5B
:1039D0008093C12A089580911628909117284091CC
:1039E000462A5091472A6091482A7091492A97FDAA
:1039F000019695958795092E000CAA0BBB0B4817CD
:103A000059076A077B0750F08091C32A9091C42A16
:103A1000892B21F01092C32A1092C42A08954F9244
:103A20005F926F927F928F929F92AF92BF92CF924E
:103A3000DF92EF92FF92CF93DF93EC016A017B015B
:103A4000488459846A847B848C809D80AE80BF804A
:103A500020E030E0A901C301B2010E94B5518823E2
:103A6000A1F1A5019401C701B6010E9448510E942D
:103A70002C529B0177FF04C022273327261B370BCC
:103A8000B901330F880B990B0E9464529B01AC0162
:103A9000C301B2010E94B55187FF17C0CC82DD82FD
:103AA000EE82FF826C817D818E819F81DF91CF913B
:103AB000FF90EF90DF90CF90BF90AF909F908F904E
:103AC0007F906F905F904F900895488059806A80F2
:103AD0007B80A301920160E070E080E89FE30E9498
:103AE0004851A50194010E9471534B015C01A7014B
:103AF0009601C301B2010E9471539B01AC01C50143
:103B0000B4010E9449516C837D838E839F83CACF09
:103B10008550883070F4E82FF0E0EF56F24E0C94A8
:103B2000A955A41DAC1DB41DBC1DC41DCC1DD41DA8
:103B3000DC1D60937E2870937F286CE87EE184E032
:103B40000E94310481E00895609380287093812859
:103B500066E87EE185E0F4CF609382287093832845
:103B600060E87EE186E0ECCF60938428709385283E
:103B70006AE77EE187E0E4CF609386287093872828
:103B800064E77EE188E0DCCF609388287093892821
:103B90006EE67EE189E0D4CF60938A2870938B280B
:103BA00068E67EE18AE0CCCF60938C2870938D2804
:103BB00062E67EE18BE0C4CF60938E2870938F28FD
:103BC0006CE57EE18CE0BCCFDC01ED91FD91808164
:103BD000ED91FD919081ED91FD916C9163708E233B
:103BE00009F064609F2309F06860E1E0FEE1E60F00
:103BF000F11D659565956D936D917D918D919D916B
:103C0000099423C01AC012C016C010C01EC009C03B
:103C100014C013C006C019C009C00DC007C00DC034
:103C200014C062507040804090400BC061507040A2
:103C30008040904006C06E5F01C06F5F7F4F8F4F26
:103C40009F4F9E938E937E936E9308958091A028AC
:103C50009091A1280C94E41D80919E2890919F281A
:103C60000C94E41D80919C2890919D280C94E41D57
:103C700080919A2890919B280C94E41D809198281B
:103C8000909199280C94E41D809196289091972802
:103C90000C94E41D80919428909195280C94E41D37
:103CA00080919228909193280C94E41D8091902803
:103CB000909191280C94E41D80918E2890918F28EA
:103CC0000C94E41D80918C2890918D280C94E41D17
:103CD00080918A2890918B280C94E41D80918828EB
:103CE000909189280C94E41D8091862890918728D2
:103CF0000C94E41D80918428909185280C94E41DF7
:103D000080918228909183280C94E41D80918028D2
:103D1000909181280C94E41D80917E2890917F28B9
:103D20000C94E41D80917C2890917D280C94E41DD6
:103D300080917A2890917B280C94E41D80917828BA
:103D4000909179280C94E41D8091762890917728A1
:103D50000C94E41DCF93DF93EC018B85823060F4EB
:103D6000F894CE010E94E41D6F81788589859A853B
:103D70007894DF91CF910895F894F6CF0F931F9325
:103D8000CF93DF93EC01062F142F70E060E0802FBB
:103D90000E94190761E070E0802F0E94140770E014
:103DA00060E0812F0E94190761E070E0812F0E947E
:103DB0001407802F90E0FC01E654F041A081A6306A
:103DC00008F04EC020E2A29FD0011124BC5F9D01EB
:103DD000285F3F4F2883398380569041FC01408102
:103DE0004C83812F90E0FC01E654F041E08170E0CB
:103DF00060E0E63030F420E2E29FF0011124BF01E0
:103E00007C5F9B01285F3F4F2A833B838056904114
:103E1000FC0130813D831F82188619861A868BE348
:103E20009FE10197F1F718962C91242381E009F482
:103E300080E0FB019085932309F082608E83BE01B0
:103E4000802F0E94881D8B87BE01812F0E94881DB4
:103E50009B85890F8B87DF91CF911F910F910895DB
:103E6000B0E0A0E0B4CF8F929F92AF92BF920F9339
:103E70001F93CF93DF93CDB7DEB7A197CDBFDEBF42
:103E800019A2423008F44AE08E010F5D1F4F842EC4
:103E9000912CB12CA12CA50194010E941751E62F61
:103EA000B901CA01EA302CF5E05DD801EE938D012D
:103EB000232B242B252B79F790E080E0109769F0D5
:103EC000FD0101900020E9F73197AF014A1B5B0B20
:103ED000BD0184EC9DE20E941609A196CDBFDEBF14
:103EE000DF91CF911F910F91BF90AF909F908F90D6
:103EF0000895E95CDACFCF92DF92EF92FF92CF93F1
:103F0000DF936B017C016DE284EC9DE20E941B1744
:103F1000EC0166277727CB016C197D098E099F0973
:103F20004AE00E94331F8C0F9D1FDF91CF91FF90BD
:103F3000EF90DF90CF900895BC01990F880B990BFB
:103F400097FD0C947B1F4AE00C94331FEF92FF9275
:103F50000F931F93CF93DF930097A9F040914728C9
:103F6000509148286091492870914A284D3D55400C
:103F70006105710544F020910028309101282F3F00
:103F80003F4F09F450C02091DD2D3091DE2D232BC1
:103F900051F42091D22D3091D32D2A5F3F4F2093A1
:103FA000D22D3093D32D2FED32E02093DD2D3093A1
:103FB000DE2D1816190624F5EC0180914728909102
:103FC0004828A0914928B0914A288D3D9540A105E7
:103FD000B10584F1E0901329F09014290FE310E06B
:103FE00028E330E048E350E066EB70E084EC9DE2CB
:103FF0000E9433128FEF9FEF809300289093012847
:104000008091DD2D9091DE2D892B49F08091D22D6C
:104010009091D32D06978093D22D9093D32D10920B
:10402000DD2D1092DE2DDF91CF911F910F91FF902A
:10403000EF90089580910028909101288C179D079A
:10404000F9F2E0901A29F0901B290FE310E028E321
:1040500030E048E350E066EB70E084EC9DE20E94C3
:1040600033128CEB90E08093D02D9093D12D8EE67F
:1040700090E08093D22D9093D32DCE010E949C1F6F
:10408000C0930028D0930128BBCFFF920F931F93BA
:10409000CF93DF93F62E2091402830914128AC0138
:1040A000421B530B2817390714F59A0180934028B7
:1040B00090934128E901219780919D2A882329F036
:1040C00070E060E080E10E94A80610E000E061E09E
:1040D00070E080E10C171D0774F40E94A80670E0E0
:1040E00060E080E10E94A8060F5F1F4FF0CF9A01A9
:1040F000285F3F4FDBCF0E94A8060E94B80760935D
:10410000992A70939A2A80939B2A90939C2AC1E0C3
:10411000C0939D2AFF2031F061E085E00E94EF040A
:10412000C0939E2A80914028909141280196DF916A
:10413000CF911F910F91FF900C94A61FCF93DF9307
:10414000EC014CE050E061E070E080EC90E00E9417
:10415000E91A1C161D062CF4CE01DF91CF910C94A8
:104160009C1FDF91CF910895009769F0FC010190A9
:104170000020E9F73197AF01481B590BBC0184ECD3
:104180009DE20C94160990E080E00895CF93DF93B0
:10419000873F2FEF920724F4DF91CF910C949C1F5F
:1041A000EC0197FF06C087E090EF0E94B420CE019B
:1041B000F3CF84E090EFCA30D105BCF786E090EFF2
:1041C000209799F789E090EFDF91CF910C94B4207C
:1041D00040EA50E062E070E090E080E00E94E91A7E
:1041E0000E9417088091E72A9091E82A8093E52A97
:1041F0009093E62A863091059CF481E190EF0E942D
:10420000B4208091E52A9091E62A8630910510F538
:10421000880F991FFC01EE5EF0418081918115C0ED
:1042200089309105A9F740EA50E062E070E090E043
:1042300080E00E94E91A86E190EF0E94B42080910C
:10424000E42A811104C082E790EF0C94B4208DE041
:1042500090EFFBCF08958F929F92AF92BF92CF9233
:10426000DF92EF92FF920F931F93CF93DF937C0126
:104270006B018A012417350710F030E020E0E901D6
:10428000219740EF50E063E070E08AE090E00E9408
:10429000E91AC7010E94B42099E1E92E9CEFF92E9A
:1042A0008091562A9091572A0E94AA1E4B01940190
:1042B00021703327232B11F594012E193F09121673
:1042C0001306DCF16E157F05C9F08FEF9FEFC80F65
:1042D000D91FD7FF35C0C00FD11F44E650E063E0BF
:1042E00070E080EA90E00E94E91AFE01EE0FFF1FE5
:1042F000EC0DFD1D808191810E94B42080915A2A8D
:1043000090915B2A0E94AB09E0915A2AF0915B2AB6
:10431000808580FD10C082FF0EC0CE01DF91CF915D
:104320001F910F91FF90EF90DF90CF90BF90AF90D3
:104330009F908F9008957401B3CF81E090E0C7CF34
:10434000C017D10754F2C01BD10BC7CFCF92DF9259
:10435000EF92FF922091A72A211156C041110EC061
:10436000C090A628D090A728E090A828F090A9286F
:10437000C616D706E806F90609F446C06B017C01AB
:10438000C092A628D092A728E092A828F092A92847
:104390004CE350E064E070E08CE390E00E94E91AA6
:1043A0008091452890914628892B79F081EBC81699
:1043B00084E0D806E104F10444F081E290EFFF903C
:1043C000EF90DF90CF900C94B420F7FE17C0C70198
:1043D000B6010E947B1F20E030E040E85FE360917F
:1043E00031287091322880913328909134280E948E
:1043F000B551882349F083E290EFE1CF4AE0C7014D
:10440000B6010E94331FE7CFFF90EF90DF90CF906F
:1044100008958F929F92AF92BF92CF92DF92EF92C8
:10442000FF920F931F93CF93DF93962E7A018823E9
:1044300061F040EA50E061E070E090E080E00E94CE
:10444000E91A85E290EF0E94B42081E2C82E88E24A
:10445000D82ED0E0C0E09AE2892E911051C0EC161F
:10446000FD0609F451C080910428909105288C170D
:104470009D0721F50FEF1FEFF601A080B18063E0EB
:1044800070E0C430D10514F462E070E04AE250E01C
:10449000CE01837099279C01829EC001839E900D5E
:1044A00011240E94E91A0093D62D1093D72D009362
:1044B000D42D1093D52DC5010E94C620219632E03F
:1044C000C30ED11CC830D10541F68FEF9FEF80930A
:1044D000D62D9093D72D8093D42D9093D52DE09207
:1044E0000428F0920528DF91CF911F910F91FF9042
:1044F000EF90DF90CF90BF90AF909F908F900895F6
:10450000EC16FD0609F0B6CF07EE19EFB5CF7F9296
:104510008F929F92AF92BF92CF92DF92EF92FF92D3
:104520000F931F93CF93DF93062F5A01882361F0D7
:1045300040EA50E061E070E090E080E00E94E91A1B
:1045400080E390EF0E94B4202FE6C22E2AE2D22E02
:10455000D0E0C0E010E03AE2732E011169C0AC1661
:10456000BD0609F469C080910228909103288C1738
:104570009D0729F5EE24EA94FE2CF60180809180B7
:1045800063E070E0C430D10514F462E070E04AE208
:1045900050E0CE01837099279C01729EC001739EEA
:1045A000900D11240E94E91AE092D62DF092D72D99
:1045B000E092D42DF092D52DC4010E94C620111195
:1045C00007C011E0F60180819181892B09F410E088
:1045D0002196F2E0CF0ED11CC830D10509F0BDCF35
:1045E0008FEF9FEF8093D62D9093D72D8093D42D6E
:1045F0009093D52D112341F0809145289091462824
:1046000011E0892B09F410E01093D12AA09202281E
:10461000B0920328DF91CF911F910F91FF90EF90FF
:10462000DF90CF90BF90AF909F908F907F90089534
:10463000AC16BD0609F09ECF87EEE82E89EFF82E66
:104640009CCF1F93CF93DF93182F8091AE2AC6E0A3
:10465000D0E081110AC080919F2AC0913C28D0915E
:104660003D28882311F0C7E0D0E08FEF9FEF8093C3
:10467000D62D9093D72D8093D42D9093D52D82E075
:104680008093D82D8093D92D40EA50E0C930D105D0
:1046900009F05DC062E070E090E080E00E94E91AFD
:1046A00086E190EF0E94B4208091E42A81114CC0F1
:1046B00082E790EF0E94B42084EB90E08093D02DAD
:1046C0009093D12DCEE1D0E0C093D22DD093D32DB5
:1046D0008DE390EF0E94B4208CEC90E08093D02D7D
:1046E0009093D12DC093D22DD093D32D8FE390EF03
:1046F0000E94B42080913E2890913F280E949E20E5
:104700001123D9F040EA50E063E070E090E080E0EF
:104710000E94E91A81E490EF0E94B42049E150E040
:1047200063E070E084E890E00E94E91A8091832AB7
:104730009091842A01960E949C1F90E080E0DF9176
:10474000CF911F910C94A61F8DE090EFB3CF61E045
:1047500070E090E080E00E94E91ACC0FDD1FCE5E91
:10476000D04188819981A6CF8091E42C9091E52C4D
:104770000297029750F4809160288823C9F150E095
:1047800040E061E081E00E9487228091D12C9091ED
:10479000D22C0297029750F480916128882389F1E6
:1047A00050E040E061E081E00E94092280916228AF
:1047B000882329F081E00E9421230E94E8201092A2
:1047C0005C2810925D2810925E2810925F2810924B
:1047D0006028109261288FEF9FEF80936328909359
:1047E0006428809365289093662810926228089523
:1047F000409165285091662857FDC7CF61E080E061
:10480000C2CF409163285091642857FDCFCF61E01B
:1048100080E0CACFCF92DF92EF92FF920F931F9367
:10482000CF93DF93EC01088119816A817B81601B42
:10483000710B072E000C880B990B0E9464529B0190
:10484000AC0160E070E080EC91E40E94BA516B0131
:104850007C0168857985601B710B072E000C880B25
:10486000990B0E9464529B01AC01C701B6010E94E2
:1048700071530E942E540E942C52CB0197FF02C00C
:104880000C96FCCF6CE070E00E949555FC01EE0F99
:10489000FF1FEA55F141808191810197DF91CF910E
:1048A0001F910F91FF90EF90DF90CF9008954F925E
:1048B0005F926F927F928F929F92AF92BF92CF92B0
:1048C000DF92EF92FF920F931F93CF93DF93CDB7B9
:1048D000DEB72E97CDBFDEBFC0903128D0903228F2
:1048E000E0903328F0903428BC0104970CF0B2C05B
:1048F0006F5F7F4F072E000C880B990B0E9464524C
:104900009B01AC0160E070E080E89FE30E94BA5137
:104910006093AA287093AB288093AC289093AD281D
:1049200020914528309146282230310561F421E05C
:104930002983A70196010E94B551811101C01982F6
:1049400039813093AE288090AA289090AB28A0900F
:10495000AC28B090AD2841E04983A7019601C5017C
:10496000B4010E94B551811101C01982598150933F
:10497000582AA7019601C501B4010E94B5518823A8
:1049800009F466C18091AE28811162C180923128FC
:1049900090923228A0923328B092342860910A284D
:1049A00070E090E080E00E946452A50194010E94B2
:1049B00071530E942C52AB018091112990911229C0
:1049C000BA010E94955580931129909312298093E2
:1049D0000B2990930C296091472870914828809169
:1049E000492890914A280E94645269837A838B8374
:1049F0009C839B01AC0160EC71EE84E69CE40E9418
:104A0000BA51A50194010E94715320E030E044EBBB
:104A100052E40E94BA510E942E540E9433526B01FC
:104A20007C010091442C1091452CD8018C918E7FF3
:104A30008C938C918670823009F470C08430D9F0E8
:104A4000811120C044E0CC0CDD1CEE1CFF1C4A95FB
:104A5000D1F718C063507109072E000C880B990B11
:104A60000E9464526093AA287093AB288093AC286C
:104A70009093AD2868CF62E0F694E794D794C794FA
:104A80006A95D1F780E090E0A1E0B0E08093522CED
:104A90009093532CA093542CB093552C97014427FA
:104AA00055272B873C874D875E872093462C309374
:104AB000472C4093482C5093492CC701B6018827B6
:104AC000992760934A2C70934B2C80934C2C909395
:104AD0004D2C232B242B252B09F444C0412C512C85
:104AE00032016394A3019201215031094109510916
:104AF0002D833E834F835887613071058105910571
:104B0000A9F4C701B6010E9417512B873C874D8736
:104B10005E874D805E806F807884E4CF53E0CC0C5C
:104B2000DD1CEE1CFF1C5A95D1F7ACCF60934A2CCC
:104B300070934B2C80934C2C90934D2C4092522C84
:104B40005092532C6092542C7092552C2B853C859E
:104B50004D855E852093462C3093472C4093482CFE
:104B60005093492C8091522C9091532CA091542C0D
:104B7000B091552C0197A109B1098093522C9093C3
:104B8000532CA093542CB093552C40914A2C509107
:104B90004B2C60914C2C70914D2C411551056105A9
:104BA000710561F0415051096109710940934A2C26
:104BB00050934B2C60934C2C70934D2C4091462C71
:104BC0005091472C6091482C7091492C40934E2C69
:104BD00050934F2C6093502C7093512C452B462BA7
:104BE000472B21F480914A2C90914B2CD8011C9694
:104BF0008D939C931D971A961D921C921B978C91D6
:104C000081608C938091452890914628892B01F5ED
:104C1000A501940169817A818B819C810E94BA519E
:104C20000E942C5240E02E96CDBFDEBFDF91CF9187
:104C30001F910F91FF90EF90DF90CF90BF90AF90BA
:104C40009F908F907F906F905F904F900C94A621D3
:104C50002E96CDBFDEBFDF91CF911F910F91FF90B8
:104C6000EF90DF90CF90BF90AF909F908F907F900C
:104C70006F905F904F9008950F931F93CF93DF93A2
:104C80008091E72A9091E82A88309105A9F440EABA
:104C900050E061E070E090E080E00E94E91A8CE46E
:104CA00090EF0E94B4201092402810924128DF918A
:104CB000CF911F910F91089510929F2A1092AE2AC2
:104CC000863091050CF04DC08091E52A9091E62A3E
:104CD00080933C2890933D2882309105D1F481E067
:104CE0008093422880E00E94212380919F2A811195
:104CF00004C08091AE2A8823D1F240EA50E062E0FD
:104D000070E090E080E0DF91CF911F910F910C94C3
:104D1000E91A049739F70CE318E2C8E0D0E00E94E2
:104D2000D04FBE010E949555D8015E962D913C91C1
:104D30005F97FC01EE0FFF1FE45BF74D80819181CF
:104D40005E968D939C935F973327208331832197C1
:104D500002501109209719F7109243281092442805
:104D6000C1CF21E08730910509F020E020939F2AF0
:104D700021E08630910509F020E02093AE2A0997C2
:104D800009F0B0CF8091E42A91E089278093E42A4A
:104D900040EA50E062E070E090E080E00E94E91AB2
:104DA00086E190EF0E94B4208091E42A81111AC01C
:104DB00082E790EF0E94B420809145289091462888
:104DC000892B61F08091E42A882349F020914528BD
:104DD0003091462881E02130310509F080E0809350
:104DE000D12A80CF8DE090EFE5CF209145283091FA
:104DF00046282230310509F04BC02091432A3091DA
:104E0000442A1216130624F48217130609F040C030
:104E1000842F90E024E0959587952A95E1F7877097
:104E2000613161F0623129F1603191F590E00196D4
:104E300080933E2890933F280C949E20863040F526
:104E400090E02091E72A3091E82A8217930701F138
:104E50008093E72A9093E82A8093E52A9093E62AA4
:104E60008091582A882319F01092582A08950C949A
:104E70003C26873069F0282F30E0843020F0C901CB
:104E800003970C94572487E090E0821B930BF9CF93
:104E90000895CF93DF9380913C2890913D288230F4
:104EA0009105E1F150F4C0913E28D0913F2821971F
:104EB0000197C1F0D0E0C0E015C0C0914C28D0915E
:104EC0004D288430910571F00597A1F70E94D04FCD
:104ED000892F990F990B60913E2870913F280E946D
:104EE0009555EC01109243281092442860E0CE01C1
:104EF0000E9445208091D12C9091D22C019702974D
:104F000088F4CC0FDD1FCF5DD74D888199818093C8
:104F1000972A9093982ADF91CF91089581E080930A
:104F20004228C8CF81E090E0F2CF0F931F93CF9338
:104F3000DF938091E42A8823A9F088E790E08093AA
:104F400016289093172881E08093452A80914B285A
:104F50008823B1F181E08093A02ADF91CF911F9146
:104F60000F9108958091E42C9091E52C0197029780
:104F700068F7C0914028D0914128CE01029608E000
:104F800010E0B8010E949555FC01EE0FFF1FE1599A
:104F9000F54D20813181265A3F4FCE010196B8014F
:104FA0000E949555FC01EE0FFF1FE159F54D8081E0
:104FB0009181281B390B2093162830931728C6CFD0
:104FC000DF91CF911F910F910C9449278091D12AA5
:104FD000811122C08091452890914628019721F4A3
:104FE0008091BF2A81110AC080914528909146285E
:104FF000029771F48091C02A882351F08091A02AF1
:10500000882359F01092A02A0E9449271092A12AC1
:105010001092BF2A1092C02A089581E08093A12A9D
:10502000F7CF0E940C57CF92DF92EF92FF920F932F
:10503000FC01C12CB9E0DB2EBDE3EB2EF12CC082CC
:10504000D182E282F3821482158281E090E086832D
:105050009783C0901128D0901228E0901328F090E8
:105060001428F694E794D794C79490E04C155D0506
:105070006E057F0540F4F694E794D794C7949F5F3C
:105080009630A1F797E004600187892F8095A82FBB
:10509000A170B0E084E0AA0FBB1F8A95E1F791628E
:1050A0009A2B80E0232B09F480E4982B90870F91B2
:1050B000FF90EF90DF90CF9008950F931F93CF93C1
:1050C000DF93CDB7DEB72A97CDBFDEBF8C01FC01E1
:1050D000878181110CC01086118612861386148672
:1050E000158616861786108A118A81E0878380913B
:1050F000E305F8019681892B8093E30561E070E078
:1051000083810E94190761E070E0F80184810E94A8
:1051100019078091C10884608093C1088091C008FC
:1051200081628093C00840915C2C50915D2C60910D
:105130005E2C70915F2C0091602C2091622C30913C
:10514000632CCE0101960E94132899858A8590933D
:10515000C0088093C1082A96CDBFDEBFDF91CF91F2
:105160001F910F910895CF92DF92EF92FF920F93CC
:105170001F93CF93DF93EC016A017B01C114D1042B
:10518000E104F10439F4C12C88E4D82E88EEE82E2D
:10519000FF24F394FE01FF96C082D182E282F38263
:1051A00081E28DAF80E28EAF369610818FA987FDA8
:1051B00009C061E070E00E94190761E070E08FA90A
:1051C0000E94140761E070E088AD0E94190761E059
:1051D00070E088AD0E9414078DA981114DC0C9A24D
:1051E000DAA2EBA2FCA2812F90E08DA39EA381E026
:1051F00090E08FA398A7812F90E0B0E0A0E089A76E
:105200009AA7ABA7BCA78F8D98A184569C4221F486
:1052100084E69CE20E945D288EA987FD86C061E03D
:1052200070E00E94190761E070E08EA90E941407E7
:1052300064E670E080E090E00E94E70770E060E0E4
:105240008EA90E94140764E670E080E090E00E945E
:10525000E70761E070E08EA90E94140768EC70E037
:1052600080E090E0DF91CF911F910F91FF90EF9040
:10527000DF90CF900C94E7070AEB1FEEF12C813002
:10528000E1F461E070E08AA50E94190770E060E037
:105290008AA50E94140761E070E08CA50E9419079E
:1052A00070E060E08CA50E9414078BA587FDB4CF49
:1052B00070E060E00E941907AFCFF80181918F0183
:1052C000863080F5F0E28F9FC00111249C5F049628
:1052D0002F8D38A12817390751F461E070E08F2D28
:1052E0000E94190770E060E08F2D0E941407F3946C
:1052F00026E1F212E2CF61E070E08EA50E9419076C
:1053000061E070E08EA50E9414078FA587FD84CF11
:1053100061E070E00E94190761E070E08FA50E94D3
:1053200014077ACF90E080E0D2CFDF91CF911F9128
:105330000F91FF90EF90DF90CF9008955F926F9262
:105340007F928F929F92AF92BF92CF92DF92EF9215
:10535000FF920F931F93CF93DF93CDB7DEB7629782
:10536000CDBFDEBF3C010B871C872D873E87042FF6
:105370004F87588B698B7A8B29893A894B855C8555
:105380006D857E85CE0101960E94132859841A8569
:10539000D30118968C91882319F081FF18C0F894D6
:1053A0005092C0081093C1086296CDBFDEBFDF9156
:1053B000CF911F910F91FF90EF90DF90CF90BF9012
:1053C000AF909F908F907F906F905F90089580FF37
:1053D000E7CFF30182849384A484B584C12CD12CBB
:1053E0007601B0E09401A501B601C701A0E00E94DA
:1053F000DB55A9F1217030E040E050E060E070E062
:1054000080E090E00E94DB55E9F090E080E0B0336E
:1054100070F48B2F869586958695F0E28F9FC0015C
:105420001124805F9B4F2B2F2770820F911DFC0151
:10543000408193012B0F311DF901428BFC0120812A
:10544000287F20839401A501B601C70101E00E94D5
:10545000C05549015A016B017C01BF5FC3CFD30125
:105460001E968D909D90AD90BC905197C12CD12CE3
:105470007601B0E29401A501B601C701A0E00E9447
:10548000DB5509F48DCF217030E040E050E060E062
:1054900070E080E090E00E94DB55E9F090E080E071
:1054A000B03370F48B2F869586958695E0E28E9FBB
:1054B000C0011124805F9B4F2B2F2770820F911DFD
:1054C000FC01408193012B0F311DF901428BFC013E
:1054D0002081287F20839401A501B601C70101E046
:1054E0000E94C05549015A016B017C01BF5FC2CFC8
:1054F0000C948356FF920F931F93CF93DF938C01ED
:10550000EB01F8800E948450F81621F06F2DC8013D
:105510000E948C50CE01DF91CF911F910F91FF908F
:1055200008950F931F93CF93DF938C01EB010E949B
:1055300084508883C80101960E9484508983CE01DB
:10554000DF91CF911F910F910895FF920F931F93B9
:10555000CF93DF93EC018B01FB01F0800E9484501C
:10556000F81621F06F2DCE010E948C50F801F180C9
:105570002196CE010E948450F81621F06F2DCE01A5
:105580000E948C50C801DF91CF911F910F91FF9025
:105590000895CF93DF93C0E1D0E0BE016F5E774DF9
:1055A000CE010E94A52A2296C032D105B1F7DF9123
:1055B000CF910895CF93DF93C4E2D0E0BE01655B45
:1055C000754DCE010E94A52A2296C433D105B1F7AC
:1055D000DF91CF910895CF93C62F80934B282AE572
:1055E00030E0209316283093172861E0682784E084
:1055F0000E94EF0460914B2886E00E94EF04CC23C8
:1056000091F00E94952780917F2A81110E94DA2AC9
:105610008091802A81110E94C92A1092802A1092BA
:105620007F2ACF9108958091E42A882361F388E747
:1056300090E080931628909317281092452AE3CF84
:1056400090E00C948450882349F086E00E94202B3F
:1056500091E0811101C090E0909315298091152966
:105660002FE130E0882311F020E038EF20931A2951
:1056700030931B2920EE3FEF882311F02FEF3FEFEF
:105680002093182930931929811107C08AE090E0EE
:105690008093132990931429089580E090EAF8CF1D
:1056A0006F927F928F929F92AF92BF92CF92DF9232
:1056B000EF92FF920F931F93CF93DF93CDB7DEB797
:1056C000CA54D109CDBFDEBFD82E81E00E94232B62
:1056D0001092A72A70E060E084EC9DE20E94C4185A
:1056E0008091152861E0811163E084EC9DE20E94C5
:1056F000B310E0901A29F0901B290DE110E020EF83
:1057000030E050E040E070E060E084EC9DE20E9418
:1057100033128FEF9FEF8093D62D9093D72D8093E8
:10572000D42D9093D52D8CE390E08093D02D909341
:10573000D12D85E090E08093D22D9093D32D82E0FF
:105740008093D82D8093D92D87E590EF0E94B420C7
:10575000DD2009F413C28AE090E08093D02D90936D
:10576000D12D8EE190E08093D22D9093D32D82E6BF
:1057700090EF0E94B42068EE73E080E090E00E9419
:10578000E70780E1E6E2FEEEDE01D39601900D929E
:105790008A95E1F7FE01B39680E1DF011D928A95BB
:1057A000E9F77E01B3E3EB0EF11C8F013F014701E6
:1057B00040E1C42ED12CBE016D5B7F4FC6010E941B
:1057C000912A2596AEACBFAC2597D401AD92BD927F
:1057D0004D01BE016F5F7F4FC60144960E94912A22
:1057E000B1E0AB1AB10849815A81E8E0AE16B104C4
:1057F00038F481E09A01245C3F4F2937310508F0E5
:1058000080E0D3014D935D933D0181115AC084E046
:105810000E94202B91E0811101C090E090933728E5
:1058200088E00E94202B90E08093432A9093442AA2
:105830008AE00E94202B91E0811101C090E09093BA
:10584000622A8EE00E94202B90E08093162990938C
:10585000172980915C2A90915D2A0E94AB09809162
:105860005A2A90915B2A0E94AB09E0915A2AF09142
:105870005B2A808580FDFEC140EF50E062E070E071
:105880008AE090E00E94E91A87E690EF0E94B42037
:1058900080915C2A90915D2ADC0118962C9120FF62
:1058A00007C0E0915A2AF0915B2A208520FD29C08B
:1058B0000E94AB0980915A2A90915B2A0E94AB0901
:1058C000E7CFE2E0CE0ED11CF0E2CF16D10409F012
:1058D00072CFA1E2B8E24FE65AE2C7014096F70163
:1058E000219131917F012D933D93F80121913191C7
:1058F0008F01FA0121933193AF018E159F0579F73E
:1059000086CF809136EE909137EEA09138EEB0912F
:1059100039EE2B968CAF9DAFAEAFBFAF2B972091DA
:10592000372881E0282730E042E050E0BE01695B83
:105930007F4F85E790EF0E942B2121E0892B09F012
:1059400020E02093372867E378E284E090E00E942B
:105950007A2A80913AEE90913BEEA0913CEEB09184
:105960003DEE27968CAF9DAFAEAFBFAF279720918E
:10597000152930E042E050E0BE016D5B7F4F82E8C8
:1059800090EF0E942B2121E0019709F020E0209365
:10599000152965E179E286E090E00E947A2A20915B
:1059A000622A81E0282730E042E050E0BE01695BD6
:1059B0007F4F8AE890EF0E942B2121E0892B09F08C
:1059C00020E02093622A62E67AE28AE090E00E9478
:1059D0007A2A2091152881E0282730E042E050E023
:1059E000BE01695B7F4F86E990EF0E942B2121E089
:1059F000892B09F020E02093152865E178E28CE0FE
:105A000090E00E947A2A209116293091172943E0CC
:105A100050E06BE078E282EA90EF0E942B218093C5
:105A200016299093172966E179E28EE090E00E94B2
:105A3000A52A809116299091172963E070E00E94B1
:105A40009555FC01EE0FFF1FE056F14180818093D8
:105A50000A2882E2EEE3FEEEDE01119601900D923D
:105A60008A95E1F72091432A3091442A41E150E0A0
:105A7000BE016F5F7F4F88EA90EF0E942B218093D9
:105A8000432A9093442A63E47AE288E090E00E94FB
:105A9000A52A80E00E94502BBE016D5B7F4F90E0F5
:105AA00080E00E94912A25968EAD9FAD259718160D
:105AB000190624F48093082890930928BE016F5F8B
:105AC0007F4F82E090E00E94912A89819A81181686
:105AD000190624F4809306289093072887E190E024
:105AE0000E94E755FC01209106283091072840913B
:105AF0000828509109288FEF9FEF83879487858727
:105B00009687838B948B88E090E0858B968B40837F
:105B10005183228333831086118682E090E0848350
:105B2000958384E190E086839783E093AC2AF09399
:105B3000AD2AE091602AF091612AF89417821086CC
:105B4000118612867894E091562AF091572AF8949B
:105B50001782108611861286789487E090E08093F1
:105B6000542A9093552A8091432A9091442A8093F5
:105B70009B2D90939C2D80E00E94232B1092D02D82
:105B80001092D12D04E510E00093D22D1093D32D67
:105B900081EE90EF0E94B4201092D02D1092D12D62
:105BA0008FE690E08093D22D9093D32D8DEE90EFE1
:105BB0000E94B42080E00E94212380913E28909191
:105BC0003F280E949E2084E890E08093D02D9093FF
:105BD000D12D0093D22D1093D32D88E090E00E9418
:105BE0009C1F8FEF9FEF80934528909346280E943B
:105BF000512FE0901A29F0901B2903E410E02CE3C8
:105C000030E046E350E064EB70E084EC9DE20E94FB
:105C10003312E0901829F09019292CE330E046E384
:105C200050E064EB70E084EC9DE20E94ED17E090A0
:105C30001829F090192901E410E02AE330E047E345
:105C400050E065EB70E084EC9DE20E94ED17C65BCE
:105C5000DF4FCDBFDEBFDF91CF911F910F91FF903E
:105C6000EF90DF90CF90BF90AF909F908F907F90FC
:105C70006F900895E0915C2AF0915D2A808580FD07
:105C80000BCF40EF50E061E070E090E080E00E94D8
:105C9000E91A81EB90EF0E94B42080915C2A9091E8
:105CA0005D2AFC01208520FF07C0E0915A2AF0916F
:105CB0005B2A208520FD09C00E94AB0980915A2AE9
:105CC00090915B2A0E94AB09E8CF1092D02D1092E0
:105CD000D12D89E3E82EF12CE092D22DF092D32D34
:105CE0008BEB90EF0E94B42060ED77E080E090E0D5
:105CF0000E94E70784E10E9496070FEF13E09801E6
:105D0000281B390B25962EAF3FAF259798E7C92E54
:105D1000D12CC092D02DD092D12DE092D22DF092E4
:105D2000D32D83EC90EF0E94B42025968EAD9FADCD
:105D300025970E949C1F88EC90EF0E94B42068EE8B
:105D400073E080E090E00E94E7071092D02D10925F
:105D5000D12D24E5E22EF12CE092D22DF092D32D1C
:105D60008AEC90EF0E94B42060ED77E080E090E054
:105D70000E94E70784E10E949607D801A81BB90B8F
:105D8000CD01A983BA83C092D02DD092D12DE092BB
:105D9000D22DF092D32D0E949C1F25968EAD9FADE3
:105DA00025978D599F4F29813A8182179307DCF0FF
:105DB00084E10E949607F801E81BF90BE983FA8356
:105DC00044E650E063E070E088E790E00E94E91A62
:105DD00089819A810E949C1F64E670E080E090E0D7
:105DE0000E94E707DACF88E790E08093D02D909368
:105DF000D12D8FE690E08093D22D9093D32D82ED1C
:105E000090EF0E94B4201092D02D1092D12D8AE8EC
:105E100090E08093D22D9093D32D25968EAD9FAD9B
:105E2000259784389340C4F589819A81883E9340B0
:105E30009CF585ED90EF0E94B42025968EAD9FAD28
:105E40002597809308289093092889819A818093C7
:105E500006289093072868E078E290E080E00E94AE
:105E6000A52A66E078E282E090E00E94A52A68EB2D
:105E70007BE080E090E00E94E707F12CE12C07E84E
:105E800010E020EF30E04CE150E070E060E084ECA6
:105E90009DE20E94331200CE8AED90EF0E94B42062
:105EA000E6CFEF92FF920F931F938FE00E94960729
:105EB000893E23E0920774F4833523E092070CF0C7
:105EC00077C0853691050CF076C01F910F91FF9039
:105ED000EF90089581E090E0209145283091462888
:105EE0002817390791F3809345289093462860E05E
:105EF00087E00E94EF0470E060E080E10E94A80665
:105F0000F12CE12C0BE110E028E730E04CE650E00A
:105F10006CE370E084EC9DE20E94331288E790E02D
:105F20008093D02D9093D12D8FE690E08093D22D49
:105F30009093D32D809145289091462881309105EA
:105F400009F45AC0D8F1029709F45BC00E94131BF0
:105F50008091452890914628892B61F08091E42A10
:105F6000882349F0209145283091462881E021304E
:105F7000310509F080E08093D12A80913728882369
:105F800009F4A3CF0E9417086093A82A7093A92A46
:105F90008093AA2A9093AB2A8091A72A882309F498
:105FA00094CF80E01F910F91FF90EF900C94502BB5
:105FB00082E090E091CF90E080E08ECF80E291EFA0
:105FC0000E94B42060914728709148288091492808
:105FD00090914A280E9464522091312830913228B1
:105FE00040913328509134280E94BA510E942C527B
:105FF00041E00E94A621AACF85E291EF0E94B42041
:10600000A5CF8AE291EFFACF4F925F926F927F9283
:106010008F929F92AF92BF92CF92DF92EF92FF92B8
:106020000F931F93CF93DF93CDB7DEB72E97CDBFDE
:10603000DEBF8091452890914628019709F088C1DC
:1060400082E00E94EF0621E030E0892B11F030E081
:1060500020E02093C32A3093C42A82E00E94EF06F6
:10606000019709F475C12091D12A298381E0822703
:106070008093BF2A0E94B8074B015C01398133230A
:1060800009F42EC180910D2990910E29A0910F291C
:10609000B0911029A5019401281B390B4A0B5B0B09
:1060A000CA01B9010E94625269837A838B839C83FF
:1060B00020E030E044EB52E40E94BA5120E030E0AE
:1060C00040E05FE30E9449510E942C526B01770F20
:1060D000EE08FF080091442C1091452CD8018C91BA
:1060E0008E7F8C938C918670823009F45FC08430EF
:1060F00051F081110FC044E0CC0CDD1CEE1CFF1CE4
:106100004A95D1F707C062E0F694E794D794C79414
:106110006A95D1F780E090E0A1E0B0E08093522C46
:106120009093532CA093542CB093552C9701442753
:1061300055272B873C874D875E872093462C3093CD
:10614000472C4093482C5093492CC701B60188270F
:10615000992760934A2C70934B2C80934C2C9093EE
:106160004D2C232B242B252B09F444C0412C512CDE
:1061700032016394A301920121503109410951096F
:106180002D833E834F8358876130710581059105CA
:10619000A9F4C701B6010E9417512B873C874D8790
:1061A0005E874D805E806F807884E4CF53E0CC0CB6
:1061B000DD1CEE1CFF1C5A95D1F7ACCF60934A2C26
:1061C00070934B2C80934C2C90934D2C4092522CDE
:1061D0005092532C6092542C7092552C2B853C85F8
:1061E0004D855E852093462C3093472C4093482C58
:1061F0005093492C8091522C9091532CA091542C67
:10620000B091552C0197A109B1098093522C90931C
:10621000532CA093542CB093552C40914A2C509160
:106220004B2C60914C2C70914D2C41155105610502
:10623000710561F0415051096109710940934A2C7F
:1062400050934B2C60934C2C70934D2C4091462CCA
:106250005091472C6091482C7091492C40934E2CC2
:1062600050934F2C6093502C7093512C452B462B00
:10627000472B21F480914A2C90914B2CD8011C96ED
:106280008D939C931D971A961D921C921B978C912F
:1062900081608C93C501B4010E9462526B017C0144
:1062A00020E030E040EC5FE369817A818B819C8162
:1062B0000E9471539B01AC01C701B6010E94495174
:1062C00020E030E04AE754E40E94BA510E94335281
:1062D0006093CD2A7093CE2A8093CF2A9093D02AB0
:1062E00080920D2990920E29A0920F29B092102928
:1062F0008091AE2A811104C08091BF2A882341F188
:1063000080913728882321F10E9417086093A82ADA
:106310007093A92A8093AA2A9093AB2A8091A72AE6
:106320008823B1F080E02E96CDBFDEBFDF91CF9104
:106330001F910F91FF90EF90DF90CF90BF90AF90A3
:106340009F908F907F906F905F904F900C94502B08
:106350002E96CDBFDEBFDF91CF911F910F91FF90A1
:10636000EF90DF90CF90BF90AF909F908F907F90F5
:106370006F905F904F9008950E9417086093A32A32
:106380007093A42A8093A52A9093A62A8091852AA7
:106390009091862A63E070E00E949555892B01F563
:1063A00064EF71E080E090E00E94E70770E060E059
:1063B00084EC9DE20E94C41864EF71E080E090E0FC
:1063C0000E94E7070E942C5023E030E040E050E0BC
:1063D0000E94B4506E5F7F4F6093192870931A2803
:1063E0000E942C5023E030E040E050E00E94B45086
:1063F0006093952A7093962A0E942C5022E330E0F5
:1064000040E050E00E94B450FB014091872A509137
:10641000882A4115510509F47CC04330510509F41F
:1064200078C02091CC2D3091CD2D261B370B209399
:10643000892A30938A2A4230510534F0E091CE2DDA
:10644000F091CF2DE61BF70BE0938B2AF0938C2A6B
:106450002091CC2D3091CD2D4230510514F430E0F7
:1064600020E02093932A3093942A4115510529F076
:1064700030E020E04330510521F42091CE2D3091C1
:10648000CF2D20938F2A3093902A2091CC2D3091BC
:10649000CD2D4230510514F030E020E02093912AB8
:1064A0003093922A4115510539F04330510599F145
:1064B0004091CE2D5091CF2D40938D2A50938E2A0E
:1064C0000E942C502DE730E040E050E00E94B45094
:1064D000675E7F4F8F4F9F4F0E94645220E030E0F5
:1064E00048E452E40E94BA5160931D2870931E281C
:1064F00080931F28909320280E942C502FEF3FEF6D
:1065000040E050E00E94B45060931B2870931C2818
:1065100008959B018CCF50E040E0CECF3F924F9248
:106520005F926F927F928F929F92AF92BF92CF9223
:10653000DF92EF92FF920F931F93CF93DF93CDB72C
:10654000DEB72A97CDBFDEBF8091452890914628BF
:10655000029709F059C34423F9F08091452890919E
:106560004628029709F050C360E080E02A96CDBF2C
:10657000DEBFDF91CF911F910F91FF90EF90DF90E1
:10658000CF90BF90AF909F908F907F906F905F90D3
:106590004F903F900C94EB2A662369F18091452837
:1065A00090914628029709F02FC30E94131B8FEF8A
:1065B0009FEF809311299093122980930B29909338
:1065C0000C2961E081E00E94EB2A2A96CDBFDEBF54
:1065D000DF91CF911F910F91FF90EF90DF90CF90BF
:1065E000BF90AF909F908F907F906F905F904F90F3
:1065F0003F900C94301B222389F080914528909184
:106600004628029709F000C30E94131B8FEF9FEFEB
:10661000809311299093122960E0D4CF80911129A1
:1066200090911229019680931129909312298091BB
:106630000B2990910C29019680930B2990930C299A
:106640002091092930910A292F5F3F4F29873A87E6
:106650002093092930930A290E94B8076B017C0115
:1066600080900D2990900E29A0900F29B0901029AC
:1066700081149104A104B10409F4BDC08C149D04DB
:10668000AE04BF0408F0B7C04090382850903928B5
:1066900060903A2870903B2860910A2870E090E062
:1066A00080E00E946452209131283091322840913C
:1066B0003328509134280E9471539B01AC0160E053
:1066C00070E68AE697E40E94BA5169837A838B83E5
:1066D0009C83C701B6010E9462526D837E838F83C3
:1066E0009887C501B4010E9462529B01AC016D8183
:1066F0007E818F8198850E9448519B01AC01698100
:106700007A818B819C810E94BA5120E030E04AE777
:1067100054E40E9471534B015C01809107299091D0
:106720000829FC01EE0FFF1FEE0FFF1FE552F74D8A
:1067300080829182A282B38201966BE070E00E9417
:106740009555809307299093082989859A850B97F9
:106750001CF18CE2EBEDF8E2AFEAB8E201900D92A9
:106760008A95E1F729ED3AE144E050E06BE070E012
:106770008FEA98E20E94174E8091C3289091C42816
:10678000A091C528B091C6288093382890933928C5
:10679000A0933A28B0933B28A30192016091382836
:1067A0007091392880913A2890913B280E94485155
:1067B0000E942C529B0177FF04C022273327261BFF
:1067C000370BB901330F880B990B0E946452A30158
:1067D00092010E94BA5120E030E040E85EE30E945E
:1067E0006C53181644F48092382890923928A0925D
:1067F0003A28B0923B28C0920D29D0920E29E092FF
:106800000F29F09210294090382850903928609034
:106810003A2870903B28B301A2018EEB9CE20E94C3
:106820000F1D0E942E5469837A838B839C83009171
:106830000A2810E0B801012E000C880B990B0E9469
:1068400064526B017C0120913128309132284091B3
:106850003328509134280E9471530E942E540E9474
:106860002C526D837E832091E42A222319F13090EB
:10687000452A072E000C880B990B0E9464524B018D
:106880005C018D819E8163E070E00E949555072E2A
:10689000000C880B990B0E9464529B01AC01C5014E
:1068A000B401332009F49CC00E9449510E942C522B
:1068B0006D837E838091112990911229ED81FE8153
:1068C0008E179F0709F0B5C18091452A91E089276D
:1068D0008093452A10921129109212298091AE2896
:1068E000882309F44BC180910B2990910C29B801A0
:1068F0000E949555892B09F041C11092AE28109243
:106900000B2910920C298090AA289090AB28A09077
:10691000AC28B090AD288092312890923228A09275
:106920003328B092342880914528909146280297C8
:1069300009F059C0A7019601C301B2010E94715329
:1069400020E030E040EC51E40E94BA510E942E5405
:106950000E942C5240E00E94A6216091472870912D
:1069600048288091492890914A280E9464529B01AE
:10697000AC0160EC71EE84E69CE40E94BA51209177
:1069800031283091322840913328509134280E9488
:10699000715320E030E044EB52E40E94BA510E946F
:1069A0002E540E9433526B017C012091442C309173
:1069B000452C2D833E83F90180818E7F80838081E9
:1069C0008670823009F46DC0843019F1811128C0BD
:1069D000A4E0CC0CDD1CEE1CFF1CAA95D1F720C056
:1069E0000E94485163CF8091452890914628892B79
:1069F00009F0B3CF609147287091482880914928C9
:106A000090914A280E946452A50194010E94BA51B3
:106A10009FCF12E0F694E794D794C7941A95D1F7D4
:106A200080E090E0A1E0B0E08093522C9093532C52
:106A3000A093542CB093552C9701442755272093AD
:106A4000462C3093472C4093482C5093492CC70137
:106A5000B6018827992760934A2C70934B2C80931A
:106A60004C2C90934D2C2115310541055105C9F150
:106A7000412C512C3201639453014201F1E08F1AF1
:106A80009108A108B108613071058105910589F46B
:106A9000C701B601A50194010E94175124013501D7
:106AA000EBCFB3E0CC0CDD1CEE1CFF1CBA95D1F78C
:106AB000B7CF60934A2C70934B2C80934C2C9093BF
:106AC0004D2C4092522C5092532C6092542C709228
:106AD000552C2093462C3093472C4093482C5093B0
:106AE000492C8091522C9091532CA091542CB09110
:106AF000552C0197A109B1098093522C9093532CE6
:106B0000A093542CB093552C40914A2C50914B2C6F
:106B100060914C2C70914D2C41155105610571050A
:106B200061F0415051096109710940934A2C509319
:106B30004B2C60934C2C70934D2C4091462C5091D3
:106B4000472C6091482C7091492C40934E2C5093C7
:106B50004F2C6093502C7093512C452B462B472B78
:106B600021F480914A2C90914B2CED81FE818487F9
:106B700095871286138680818160808380910D299C
:106B800090910E29A0910F29B0911029892B8A2B61
:106B90008B2B79F169817A818B819C810E942C52A7
:106BA0006B017C018091BD2A9091BE2A092E000CB8
:106BB000AA0BBB0BC816D906EA06FB06D1F0A091BA
:106BC0000A28B0E0A70196010E94D35028E130E0E6
:106BD00040E050E00E94B450CA01B9010E946452E2
:106BE0000E942C5240E00E94A621C092BD2AD09261
:106BF000BE2A80914B2881110E94301B81E090E0D9
:106C00008093C32A9093C42A2A96CDBFDEBFDF911A
:106C1000CF911F910F91FF90EF90DF90CF90BF9099
:106C2000AF909F908F907F906F905F904F903F902C
:106C300008952D813E8137FF04C02F5F3F4F2D8384
:106C40003E83ED81FE81F595E795E817F907E4F6B7
:106C50001092C32A1092C42AD7CF1F920F920FB658
:106C60000F9211242F933F934F935F936F937F93D2
:106C70008F939F93AF93BF934091D82A5091D92A75
:106C80006091DA2A7091DB2A8091D62A9091D72AD6
:106C90002091D42A3091D52A420F531F611D711DB6
:106CA0002091D22A3091D32A820F931F883E23E06D
:106CB000920730F0885E93404F5F5F4F6F4F7F4F7A
:106CC0008093D62A9093D72A4093D82A5093D92AD2
:106CD0006093DA2A7093DB2A8091E02A9091E12A6E
:106CE000A091E22AB091E32A0196A11DB11D8093E3
:106CF000E02A9093E12AA093E22AB093E32A81E06C
:106D00008093B60ABF91AF919F918F917F916F91C0
:106D10005F914F913F912F910F900FBE0F901F9059
:106D200018951F920F920FB60F9211242F933F9335
:106D30004F935F936F937F938F939F93AF93BF9383
:106D4000EF93FF9385E00E944309FF91EF91BF917C
:106D5000AF919F918F917F916F915F914F913F91F3
:106D60002F910F900FBE0F901F9018951F920F92AA
:106D70000FB60F9211242F933F934F935F936F930E
:106D80007F938F939F93AF93BF93EF93FF9384E091
:106D90000E944309FF91EF91BF91AF919F918F9115
:106DA0007F916F915F914F913F912F910F900FBE07
:106DB0000F901F9018951F920F920FB60F921124EB
:106DC0002F933F934F935F936F937F938F939F93F3
:106DD000AF93BF93EF93FF9383E00E944309FF912A
:106DE000EF91BF91AF919F918F917F916F915F9143
:106DF0004F913F912F910F900FBE0F901F901895BC
:106E00001F920F920FB60F9211242F933F934F931F
:106E10005F936F937F938F939F93AF93BF93EF9302
:106E2000FF9382E00E944309FF91EF91BF91AF91E0
:106E30009F918F917F916F915F914F913F912F9192
:106E40000F900FBE0F901F9018951F920F920FB6C4
:106E50000F9211242F933F934F935F936F937F93E0
:106E60008F939F93AF93BF93EF93FF9381E00E9423
:106E70004309FF91EF91BF91AF919F918F917F91C6
:106E80006F915F914F913F912F910F900FBE0F9097
:106E90001F9018951F920F920FB60F9211242F93E7
:106EA0003F934F935F936F937F938F939F93AF9392
:106EB000BF93EF93FF9380E00E944309FF91EF910E
:106EC000BF91AF919F918F917F916F915F914F9102
:106ED0003F912F910F900FBE0F901F9018951F920A
:106EE0000F920FB60F9211242F933F934F935F93FE
:106EF0006F937F938F939F93AF93BF93EF93FF9382
:106F000084EF9CE20E948D05FF91EF91BF91AF91BC
:106F10009F918F917F916F915F914F913F912F91B1
:106F20000F900FBE0F901F9018951F920F920FB6E3
:106F30000F9211242F933F934F935F936F937F93FF
:106F40008F939F93AF93BF93EF93FF9384EF9CE254
:106F50000E947C09FF91EF91BF91AF919F918F911A
:106F60007F916F915F914F913F912F910F900FBE45
:106F70000F901F9018951F920F920FB60F92112429
:106F80002F933F934F935F936F937F938F939F9331
:106F9000AF93BF93EF93FF9389EA9BE20E948D0525
:106FA000FF91EF91BF91AF919F918F917F916F91E1
:106FB0005F914F913F912F910F900FBE0F901F90B7
:106FC00018951F920F920FB60F9211242F933F9393
:106FD0004F935F936F937F938F939F93AF93BF93E1
:106FE000EF93FF9389EA9BE20E947C09FF91EF9166
:106FF000BF91AF919F918F917F916F915F914F91D1
:107000003F912F910F900FBE0F901F9018951F92D8
:107010000F920FB60F9211242F933F934F935F93CC
:107020006F937F938F939F93AF93BF93EF93FF9350
:1070300080914E2C90914F2CA091502CB091512CBE
:107040000197A109B10980934E2C90934F2CA093E6
:10705000502CB093512C181619061A061B063CF139
:10706000892B8A2B8B2BB9F18091462C9091472C40
:10707000A091482CB091492C0097A105B10591F041
:1070800080934E2C90934F2CA093502CB093512C66
:10709000E091442CF091452C8091522C9091532CEE
:1070A00084879587E091562CF091572C099581E0C3
:1070B0008093A60AFF91EF91BF91AF919F918F911D
:1070C0007F916F915F914F913F912F910F900FBEE4
:1070D0000F901F90189540914A2C50914B2C609125
:1070E0004C2C70914D2C4115510561057105A9F08D
:1070F000E091442CF091452C4487558782859385F7
:10710000B0E0A0E084179507A607B70784F2809146
:10711000522C9091532C848795878091462C909186
:10712000472CA091482CB091492C80934E2C9093E1
:107130004F2CA093502CB093512CB4CF1F920F9290
:107140000FB60F9211242F933F934F935F936F933A
:107150007F938F939F93AF93BF93CF93EF93FF93BF
:10716000C091AB08C2FF0AC01092362A1092352A8D
:107170001092342A84E00E94450C14C0C6FF2FC030
:107180008091332A813051F48091362AE091312A5E
:10719000F091322A90E009951092332AC0FF14C072
:1071A0000E94550CFF91EF91CF91BF91AF919F91AC
:1071B0008F917F916F915F914F913F912F910F90A0
:1071C0000FBE0F901F90189580E48093AB0881E06C
:1071D0000E94450C8091AB0885FFE4CFE1CFC7FF4B
:1071E0005CC0C3FF08C01092362A1092352A109254
:1071F000342A83E0C0CF8091A90880668093A908D3
:107200008091AB0881FF2CC08091352A882349F0FA
:107210008091AB0884FF05C082E08093AA0881E0DA
:10722000AACF9091352A8091342A9817A8F4E0913A
:10723000352A80912C2A90912D2AE80FF92FF11DE3
:1072400080818093AD088091352A8F5F8093352AA5
:1072500083E08093AA08A6CF82E08093AA088BCF10
:107260009091362A8091302A981790F48091AD0839
:10727000E091362A20912E2A30912F2AE20FF32F07
:10728000F11D80838091362A8F5F8093362AE0CF6C
:1072900086E08093AA0882E06ECF85E06CCF1F92D3
:1072A0000F920FB60F9211242F933F938F939F93BA
:1072B000EF93FF938091A508982F9C70E1F0809147
:1072C000A50894E082FF93E09093412A8093A5085B
:1072D00081E090E08093372A9093382A1092422AD6
:1072E000FF91EF919F918F913F912F910F900FBE42
:1072F0000F901F90189586FF4EC020913E2A9091C6
:107300003D2A8091A50884FF15C080913A2A8823E0
:1073100079F083E08093A40885E08093412A10925D
:10732000422A81E090E08093372A9093382AD8CF80
:1073300081E0F0CF80913C2A821790F4E0913C2AC2
:1073400080913F2A9091402AE80FF92FF11D80810A
:107350008093A80880913C2A8F5F80933C2AC0CFFD
:1073600080913B2A891760F484E090E08093372A6B
:107370009093382A8091392A81608093A708B0CFF2
:1073800080913A2A882329F083E08093A40881E041
:10739000C4CF81E0FACF87FF40C090913B2A809113
:1073A0003D2A9817D8F48091A808E0913B2A2091B3
:1073B0002A2A30912B2AE20FF32FF11D808380912E
:1073C0003B2A8F5F80933B2A90913D2A80913B2AF4
:1073D0008917D8F482E08093A40882CF80913A2A5A
:1073E000882389F087E08093A40882E08093412A73
:1073F0001092422A81E090E08093372A9093382AB5
:1074000010923D2A6DCF85E0EECF80913A2A8823F5
:1074100011F087E0BACF85E0B8CF86E07ECFCF927B
:10742000DF92EF92FF920F931F93CF93DF93A4EF1E
:10743000BCE212961D921C92139788EEC82E83E030
:10744000D82EE12CF12C1496CD92DD92ED92FC9287
:10745000179784E49FEE8D939C93119720E238E078
:107460001C962D933C931D971E961C921E9721E00F
:107470001F962C931F9734E050963C93509752964A
:107480001C92529753961C92539754961C92549761
:1074900055961C9255973BE156963C9356975796B6
:1074A0001C92579758961C92589710928D2D1092B7
:1074B0008E2DE9EAFBE212821382C482D582E68233
:1074C000F7828083918380E698E08487958788E1BE
:1074D000868789E1878780E4808B128A138A148AE1
:1074E000158A86E2868B178A108E1092422C109293
:1074F000432CE4E4FCE280E89AE0808391831282EA
:107500001382148215824AE050E060E070E0468306
:1075100057836087718712861386148615864FEF0E
:107520005FEF60E070E046875787608B718BECE51A
:10753000FCE240E059E06DE370E0408351836283F8
:1075400073831482158241E050E046835783C4E67A
:10755000DCE28EE59FEE888399831F8262E06E8372
:107560008CE08A838DE08C838BE08B8338E03D83D5
:1075700084EB9DE2FC0112821382C482D582E682F2
:10758000F7820CE71FEE00831183E4ECFDE2128228
:10759000138270EFE72EF12CE482F58200E411E013
:1075A00006831783E086F18602871387168A14867E
:1075B000158616861786258B248B0FEF1FEF028BFF
:1075C000138B008B118B278B108E118E128E15AAA8
:1075D00029E026AB2AE027AB30AF11AE12AE13AED6
:1075E00014AE15AE16AE1092032E1092042E109209
:1075F000052E1092062EC78FD0A3C4E8D4E0C58F05
:10760000D68F33AB24E234E0238F348F61AB2DEF80
:1076100022AB27EF24AB1092072E1092082E109267
:10762000092E28ED3FEE2083318310920A2E10920E
:107630000B2EE0ECFDE220E2208381839283138213
:10764000EFE8FDE2A083B1831282138214821582D7
:1076500044875587468757870E9417086093F02C08
:107660007093F12C8093F22C9093F32C0E941708C6
:10767000CDEDDCE2188219821A821B821C821D82E7
:107680001E821F82188619861A860E9417086B8729
:107690007C878D879E87ECE2EE2EFF24F394EF86A5
:1076A000F88A04E110E0098B1A8BCAECDCE218823C
:1076B00019821A821B821C821D821E821F821886DA
:1076C00019861A860E9417086B877C878D879E878C
:1076D000EF86F88A098B1A8BEEEBFCE28AE999E9CE
:1076E000A9E1BEE380839183A283B38380E090E02D
:1076F000A0EFB2E484839583A683B783E2EBFCE238
:107700004DEC5CEC6CE47DE34083518362837383D6
:1077100040E050E060E074E44483558366837783FF
:10772000E6EAFCE24AE959E969E97EE340835183EC
:107730006283738384839583A683B783DF91CF911C
:107740001F910F91FF90EF90DF90CF900895CF930E
:10775000DF93CDB7DEB7EE97CDBFDEBF88ED90E00B
:1077600084BF9093610080E094E2A4EFB0E0809346
:10777000112890931228A0931328B0931428809175
:1077800002068660809302068091000681608093E5
:107790000006809102068F7C809302068091A000F3
:1077A0008F788093A000809102068061809302060A
:1077B0001092E20581E08093E40583E08093010A62
:1077C0008FEF90E08093260A9093270A80E890E05C
:1077D0008093380A9093390A80933A0A90933B0A2F
:1077E00080933C0A90933D0A8BE08093000A80913D
:1077F000E50581608093E5058091E50582608093D1
:10780000E505E0E8FAE037E02FEF90E885E0318326
:107810002487958780837096E03C0AE0F007B9F7EB
:1078200080E094E08093DE2A9093DF2A8091DE2A24
:107830009091DF2A2FEF30E0B9010E94A0506093B1
:10784000DC2A7093DD2A8091DE2A9091DF2AE8EE0F
:10785000F3E0BF010E94A0506093D42A7093D52A10
:107860008091DE2A9091DF2ABF010E94A050809370
:10787000D22A9093D32A2093BC0A3093BD0A8091D8
:10788000B50A81608093B50A84E08093B00A809144
:10789000B00A81608093B00A78941092092E40E07B
:1078A00050E0BA0184EC9DE20E94B32888E2809304
:1078B0000B2E8093082E85E38093072E84E380931C
:1078C0000A2E87E890E080930C2E90930D2E80EF87
:1078D00090E080930E2E90930F2EE8EEF7E09490B8
:1078E000E9EEF7E09A941FEF911609F47EC0149127
:1078F0005F0122E0A20EB11C31968490082D0F7713
:1079000084EC9DE20E9413108091FB2D87FD09C03D
:10791000E091DF2DF091E02D80819091F62D89236B
:107920008083E091E12DF091E22D80819091F82DFE
:1079300089238083612F84EC9DE20E94610FE09196
:10794000E12DF091E22D80819091F72D892B80839C
:10795000F501D12CC12C10E0C016D106FCF48091A9
:10796000F92D7F01823089F48091F42D882369F00C
:10797000DF016D917D917D0184EC9DE20E941C0FE1
:10798000EFEFCE1ADE0AF701E7CFBFEFEB1AFB0AE3
:10799000649184EC9DE20E94610FF2CF8091FB2DF7
:1079A00087FD09C0E091DF2DF091E02D808190915D
:1079B000F52D892B808384EC9DE20E940210F50155
:1079C000E00FF11F87FE8ECF7F010FEFE01AF00A64
:1079D000649170E06F3F710511F464EF71E090E025
:1079E00080E00E94E707F7017DCF60E084EC9DE234
:1079F0000E94B31070E060E084EC9DE20E94C41825
:107A000082E08093D82D8093D92D8CE00E94202B8A
:107A100091E0811101C090E09093152863E08111FD
:107A200001C061E084EC9DE20E94B31081E00E94FD
:107A3000232B62E070E08FE00E94450662E070E078
:107A400084E00E94450662E070E085E00E94450601
:107A50008CE090E00E94E7558C0145E064E00E94D4
:107A6000BE1E0093602A1093612A62E070E086E0F7
:107A70000E94450682E190E00E94E755FC011282D7
:107A8000138214821582BAE0CB2ED12CC682D78203
:107A9000108612ECE12E1EEEF12EE082F182809330
:107AA0005C2A90935D2A86E0818BCF010E94140AA4
:107AB000E0915C2AF0915D2A02E310E006831783CF
:107AC00062E070E087E00E94450662E070E08CE0D2
:107AD0000E9445068CE090E00E94E7555C014CE076
:107AE00067E00E94BE1EA092562AB092572A62E01A
:107AF00070E08EE00E94450682E190E00E94E7552A
:107B0000FC011282138214821582C682D7821086EB
:107B1000E082F18280935A2A90935B2A8EE0818BD7
:107B2000CF010E94140AE0915A2AF0915B2A068341
:107B3000178384EB9DE20E94310E8091C12D9091BC
:107B4000C22DDC01ED91FC910688F789E02D609152
:107B5000C02D09958091C12D9091C22DDC01ED9130
:107B6000FC91028CF38DE02D0995882309F4DFC088
:107B700082E88093C32D61E086E00E94150561E0F4
:107B800085E00E94150561E084E00E94150561E032
:107B900087E00E94150562E082E00E94150562E020
:107BA00080E00E94150561E083E00E94150561E018
:107BB00081E00E94150582E190E00E94E755FC01FA
:107BC00012821382148215828AE090E08683978362
:107BD000108682EC9EEE80839183E0934F2AF0938F
:107BE000502A8FE0818BCF010E94140AE0914F2A26
:107BF000F091502A82E390E08683978360914B282E
:107C000011E0612784E00E94EF0460E087E00E94B9
:107C1000EF0461E083E00E94EF0461E081E00E94F4
:107C2000EF0460E086E00E94EF0460E085E00E94DF
:107C3000EF0410929E2A61E070E080E10E94450608
:107C400070E060E080E10E94A80661E070E081E100
:107C50000E94450670E060E081E10E94A80662E0B3
:107C600070E082E00E94450664E070E382E00E94DA
:107C7000310462E070E083E00E94450680EA9AE009
:107C80008093442C9093452C8091A00A8E7F809302
:107C9000A00A1093A60A1092A10A84E08093A00A79
:107CA00080E090E0A4E0B0E08093582C9093592CB1
:107CB000A0935A2CB0935B2C8091A00A8E7F809366
:107CC000A00A8091A00A8670F0E48F2EF2E49F2E25
:107CD000FFE0AF2EB12C853070F490E0FC01EE0F88
:107CE000FF1FE80FF91FEB52F14180819181A281C2
:107CF0004C01AA2EB12C950144275527C501B4018A
:107D000088279927C12CD12C7601E394B1E0CB1AB6
:107D1000D108E108F108613071058105910571F420
:107D2000C501B401A70196010E941751EFCF10922F
:107D3000C32D6FEF86E00E94AE041DCF2093462C2A
:107D40003093472C4093482C5093492C60934A2CF5
:107D500070934B2C80934C2C90934D2CC092522CB2
:107D6000D092532CE092542CF092552C6115710551
:107D70008105910561F06150710981099109609354
:107D80004A2C70934B2C80934C2C90934D2C209329
:107D90004E2C30934F2C4093502C5093512C232B2E
:107DA000242B252B21F4C0904A2CD0904B2CC09230
:107DB000AC0AD092AD0A1092AA0A1092AB0A809136
:107DC000A00A81608093A00A8FEA9CE18093562CE0
:107DD0009093572C81E08093A60A8093A50A809106
:107DE000A00A8E7F8093A00A8091A00A867090E9F5
:107DF000C92E90EDD92E93E0E92EF12C853060F458
:107E000090E0FC01EE0FFF1FE80FF91FEA53F1416C
:107E1000C080D180E280F12C80E090E0A1E0B0E071
:107E20008093522C9093532CA093542CB093552CA8
:107E30009701442755272093462C3093472C409395
:107E4000482C5093492CC701B60188279927609385
:107E50004A2C70934B2C80934C2C90934D2C2115D5
:107E600031054105510589F1412C512C32016394B2
:107E700053014201E1E08E1A9108A108B108613076
:107E800071058105910549F4C701B601A501940169
:107E90000E94175124013501EBCF4092522C509291
:107EA000532C6092542C7092552C2093462C309376
:107EB000472C4093482C5093492C60934A2C709344
:107EC0004B2C80934C2C90934D2C8091522C909164
:107ED000532CA091542CB091552C0197A109B109B4
:107EE0008093522C9093532CA093542CB093552CE8
:107EF00040914A2C50914B2C60914C2C70914D2C00
:107F0000411551056105710561F041505109610943
:107F1000710940934A2C50934B2C60934C2C7093D6
:107F20004D2C4091462C5091472C6091482C7091DB
:107F3000492C40934E2C50934F2C6093502C7093AF
:107F4000512C452B462B472B21F480914A2C9091A4
:107F50004B2C8093AC0A9093AD0A1092AA0A10920F
:107F6000AB0A8091A00A81608093A00A8FEB9AE10E
:107F70008093A22D9093A32D1092A42D1092A52D45
:107F80008EE892E38093AC2D9093AD2D85EF96E231
:107F90008093A62D9093A72D0091432A1091442AF7
:107FA00080918F2D9091902DDC01ED91FC910684B4
:107FB000F785E02D42E15AE760E070E00995109204
:107FC000912D1092922D00939B2D10939C2D0E9429
:107FD00017086093A82A7093A92A8093AA2A9093DD
:107FE000AB2A611571058105910511F00E947B5046
:107FF0008091372881110E94BC3181E00E94502B72
:1080000022242394312C0E9417086093F02C709343
:10801000F12C8093F22C9093F32C80914528909131
:1080200046286091C32A7091C42A8091C52A811183
:108030000AC081E06115710509F080E08093C22AD1
:1080400081E08093C52A8091C22A86171706A9F07D
:1080500087E00E94EF046091C32A7091C42A81E0F6
:108060006115710509F480E08093C22A80914B2844
:10807000882319F081E10E94A8068091C12A8823F3
:1080800009F48DC01092C12A80914528909146280C
:10809000892B29F08091D12A882309F46DC0209181
:1080A0001628309117286091462A7091472A8091AE
:1080B000482A9091492A032E000C440B550B0E942C
:1080C00017516093462A7093472A8093482A9093C9
:1080D000492A8091E42C9091E52C0197029708F0B1
:1080E00053C0E0914028F0914128CF010A9608E062
:1080F00010E0B8010E9495559C01220F331F2159B1
:10810000354DCF010996B8010E949555FC01EE0F3F
:10811000FF1FE159F54DD9018D919C91208131814D
:10812000821B930B865A9F4F809316289093172893
:108130008091E42A8823C1F08091452A22EE3FEF06
:10814000811102C02EE130E080911628909117280D
:10815000820F931F80931628909317288091452AA9
:1081600091E089278093452A8091A02A882379F07D
:108170001092A02A0E94492780E090E0892B09F400
:1081800042CF0E9400003CCF90E080E0CBCF8091B6
:108190004B28882389F381E08093A12AEDCF809139
:1081A000C02A882319F00E94E627E6CF8091BF2AD3
:1081B000882381F10E94E627609138287091392840
:1081C00080913A2890913B280E942E540E942C5274
:1081D0006B017C011C141D041E041F046CF68091AD
:1081E000BD2A9091BE2A8C33910554F08C199D09BB
:1081F00097FF03C091958195910903970CF4BCCF2B
:1082000040E0C701B6010E94A621C092BD2AD092CB
:10821000BE2AB2CF8091B52A81110DC00E941708E5
:108220006093B12A7093B22A8093B32A9093B42AB0
:1082300081E08093B52A4091B12A5091B22A609191
:10824000B32A7091B42A4115510561057105E1F019
:108250008091F02C9091F12CA091F22CB091F32C04
:10826000841B950BA60BB70B813D9740A105B1056B
:1082700058F080E00E9421231092B12A1092B22A75
:108280001092B32A1092B42A80918F2D9091902D44
:10829000DC01ED91FC910084F185E02D0995181623
:1082A00019060CF010C180918F2D9091902DDC015A
:1082B000ED91FC910284F385E02D0995182F87FD3F
:1082C0002FC08091912D9091922D892B49F580910D
:1082D000A02D9091A12D892B19F52091982D80E842
:1082E000820F8037E8F4822F8F7090E001968093A0
:1082F0009D2D90939E2D40919B2D50919C2D31E072
:108300004115510521F08417950709F030E03093AD
:108310009F2D207F2093972D2092912D3092922D8A
:108320008091912D9091922D8130910509F465C035
:108330008230910509F488C0892B79F5912F103F7F
:1083400008F4907F9093972D80E8890F803750F440
:108350001093982D212F2F702F5F30E020939D2DAB
:1083600030939E2D20919B2D30919C2D81E02115E5
:10837000310541F040919D2D50919E2D421753079C
:1083800009F080E080939F2D903E69F148F4903988
:1083900031F1903B41F1903859F11093962D74CF03
:1083A000983F29F0D0F386E0890F8330B0F7E09151
:1083B000AC2DF091AD2D309781F321E09B3F09F07A
:1083C00020E041E09C3F09F040E061E09A3F09F085
:1083D00060E081E0983F09F080E00995DECF2092CF
:1083E000932D3092942D2092912D3092922DD5CFB5
:1083F0001092932D1092942DF6CF8091972D803965
:1084000019F068F4803879F417FD0DC0E2E0F0E06F
:10841000E093912DF093922D1093952DBECF803B3C
:1084200039F0803E89F31092912D1092922DB5CFA4
:1084300017FDF9CF1093952DE2E08E2E912C8092AE
:10844000912D9092922DA9CF8091972D803919F07E
:10845000E8F4803841F717FDE6CF80919F2D2091F9
:10846000932D3091942D232B11F011111CC0E0910C
:10847000A42DF091A52D8823B1F23097A1F2412FC0
:108480006091952D80919D2D0995CDCF803B91F0E8
:10849000803E49F680919F2D882329F2E091A82DF6
:1084A000F091A92DEACFE091A22DF091A32D811199
:1084B000E4CFB9CF80919F2DE091A62DF091A72D0B
:1084C0008111DBCFB0CF00914F2A1091502AD801F3
:1084D00018968C9180FD13C00E941708F801C18482
:1084E000D284E384F4846C197D098E099F0960931A
:1084F0004B2A70934C2A80934D2A90934E2AC09019
:108500004B2AD0904C2AE0904D2AF0904E2AC80178
:108510000E94AB0980914A2A811116C180914F2A8D
:108520009091502A0E94A309811107C0F8ECCF1640
:10853000D104E104F1040CF407C1809137288823A9
:1085400009F4F3C00E9417086093A82A7093A92A1F
:108550008093AA2A9093AB2A8091A72A882309F4B2
:10856000E4C080E00E94502B8091AF2A9091B02A05
:1085700001968093AF2A9093B02A6BE070E00E943E
:108580009555892B99F483E00E94EF069C0191E0B8
:108590002115310509F090E080911828981731F0E5
:1085A00090931828232B11F40E9495278091AF2ACD
:1085B0009091B02A67E070E00E949555892BD1F523
:1085C0008091602A9091612A0E94AA1E6B0180907E
:1085D000E42C9090E52C12E0811A91086090D12C47
:1085E0007090D22C22E0621A710800915E2A1091DC
:1085F0005F2A0617170709F481C1CB0181709927FB
:10860000892B09F07BC180913728882309F409C19F
:108610000E9417086093A82A7093A92A8093AA2A17
:108620009093AB2A8091A72A882309F4FAC080E0AE
:108630000E94502B8091452890914628892B09F063
:1086400099C38091AF2A9091B02A6DE070E00E94AA
:1086500095558C01892B09F08DC38091672A811172
:1086600005C00E94170881E08093672A85E10E9477
:1086700096079C01265031092FA738AB60E074E0C3
:10868000681B790B072E000C880B990B263F334093
:1086900008F44FC30E9464526B017C01C092B62C57
:1086A000D092B72CE092B82CF092B92CC092632AE9
:1086B000D092642AE092652AF092662A8091622A1A
:1086C000882309F414C584E1E0E6FEEEDE01559648
:1086D00001900D928A95E1F784E1E4E7FEEEDE0178
:1086E000119601900D928A95E1F720E030E040EA82
:1086F00050E4C701B6010E94B55187FDEEC420E0E9
:1087000030E44EE754E4C701B6010E946C534E01B9
:1087100059E1850E911C18160CF0E3C3A8E88A2EC7
:10872000A3E19A2EA12CB12CDDC481E080934A2ACA
:1087300080914B288823F9F008ECC016D104E1049D
:10874000F104CCF40E94952780914A2A882309F4E9
:108750000BCFE0914F2AF091502A808580FF04CF03
:1087600010924A2A10924B2A10924C2A10924D2AAB
:1087700010924E2AF9CE11E060E081270E94EB2A88
:1087800080914B28882309F442C01092C32A10928A
:10879000C42A60E087E00E94EF0480914528909110
:1087A0004628892B59F5E091442CF091452C808185
:1087B0008E7F8083168380818E7F80831683809155
:1087C000462C9091472CA091482CB091492C809335
:1087D0004E2C90934F2CA093502CB093512C892B5E
:1087E0008A2B8B2B79F08091522C9091532C84877B
:1087F00095871286138680818160808381E08093D3
:10880000A02AA2CF80914A2C90914B2CF0CF20919E
:1088100045283091462881E02130310581F380E000
:10882000EECFC601801B910B21E030E0181619062F
:1088300014F02FEF3FEF42E08416910408F0CDC012
:108840008091832A9091842A08964091812A5091A0
:10885000822A841B950B68E070E00E949555AC015C
:10886000DC01AA0FBB1FFD01E159F54D008111810B
:10887000F80117FF07C0EE27FF27E01BF10B31952A
:10888000219531092130310549F4E531F1054CF4E8
:10889000E830F10544F52E0F3F1F0FC0E631F1051A
:1088A000FCF0C901880F991F280F391F2E0F3F1F99
:1088B0002F31310514F02EE130E017FF03C0319560
:1088C00021953109A159B54D2D933C9380914B28A9
:1088D000882361F0BA0181E090E00E9423080AC079
:1088E000E930F105C4F2220F331FD5CF61E080E0FB
:1088F0000E948722C0925E2AD0925F2A80915C2AD1
:1089000090915D2A0E94AB0980915A2A90915B2A2E
:108910000E94AB0980915C2A90915D2A0E94A30974
:10892000182F80915A2A90915B2A0E94A309B82E91
:108930001123C9F080913728882371F00E9417080D
:108940006093A82A7093A92A8093AA2A9093AB2AAD
:108950008091A72A81116BCE8091592A882309F42E
:1089600099C01092592A8091562A9091572A0E94B4
:10897000AA1E6B010091542A1091552A0617170759
:1089800009F4F9C0CB0181709927892B09F0F3C054
:1089900080913728882371F00E9417086093A82AD5
:1089A0007093A92A8093AA2A9093AB2A8091A72A30
:1089B00081113DCEC601801B910B181619060CF0D3
:1089C000AEC081E090E02091832A3091842A820F0A
:1089D000931F97FFA7C00896FCCF52E0651671045D
:1089E00008F043C08091832A9091842A0896409190
:1089F000812A5091822A841B950B68E070E00E94C6
:108A00009555AC01FC01EE0FFF1FDF01AF5DB74DC7
:108A10008D919C91280F391F29833A832D8A3E8A94
:108A2000DE0122303105D4F0119688E090E089A76C
:108A30009AA78D919C911197089714F0DE01999651
:108A4000EF5DF74D8D919C918083918380914B28B0
:108A5000882331F0BA0182E090E03FCF5596E5CF10
:108A600061E080E00E94092245CF8091E72A909141
:108A7000E82A820F931F97FF02C00A96FCCF6AE094
:108A800070E00E9495558093E72A9093E82A0E940F
:108A9000E82030CF82E088169104E0F48091832AA8
:108AA0009091842A08962091812A3091822A821BF3
:108AB000930B68E070E00E949555FC01EE0FFF1FDC
:108AC000E159F54D10821182AC0160E080E00E9416
:108AD000872249CF92E069167104E0F48091832ADD
:108AE0009091842A08962091812A3091822A821BB3
:108AF000930B68E070E00E949555FC01EE0FFF1F9C
:108B0000EF5DF74D20823182AC0160E080E00E9491
:108B1000092229CF1092582A0E943C2624CF8FEF99
:108B20009FEF51CF877099278093832A9093842A4F
:108B3000A2E08A16910408F08CC008962091812A40
:108B40003091822A821B930B68E070E00E94955559
:108B500020914B28222331F0BC0181E090E00E945B
:108B6000230805C0AC0161E080E00E948722C0922A
:108B7000542AD092552AE2E08E16910408F44CC093
:108B8000F2E06F16710408F447C080914528909177
:108B90004628019709F440C08091532A81113CC0B6
:108BA00000915A2A10915B2AD80118968C9180FD69
:108BB00033C00E941708F80101851285238534858A
:108BC000601B710B820B930B653F71408105910512
:108BD00018F181E08093532A8091512A9091522A72
:108BE0000196833091050CF06BC08093512A9093CD
:108BF000522AE091512AF091522AEE0FFF1FEE0FF8
:108C0000FF1FEC51F14160817181828193810E944B
:108C10002C52CB010E945724BB2009F40BCD80912C
:108C20003728882371F00E9417086093A82A709350
:108C3000A92A8093AA2A9093AB2A8091A72A81110E
:108C4000F6CC8091532A882309F43FC01092532A0E
:108C5000F1CCB2E06B167104C8F408962091812A19
:108C60003091822A821B930B68E070E00E94955538
:108C700020914B28222321F0BC0182E090E06FCFAD
:108C8000AC0161E080E00E94092271CF49E150E02F
:108C900063E070E084E890E00E94E91A8091832A02
:108CA0009091842A01960E949C1F8FEF9FEF8093E2
:108CB000D62D9093D72D8093D42D9093D52D57CF2B
:108CC0001092512A1092522A94CF02E080169104F9
:108CD00008F4B0CC12E06116710408F4ABCC8091BA
:108CE000832A9091842A019689839A832D8A3E8AC9
:108CF000FE010297E4F0319688E090E089A79AA7F8
:108D000080819181089714F0FE01B996808191814C
:108D100020913E2830913F288217930709F48ACC8E
:108D200080933E2890933F280E949E2083CC759686
:108D3000E3CF0E946452AB01BC0182EB9CE20E9433
:108D40000F1D6B017C012091632A3091642A4091B0
:108D5000652A5091662A0E9448510E942C529B011C
:108D600077FF04C022273327261B370B233031051A
:108D70000CF09CCC8091AF2A9091B02A6BEB70E004
:108D80000E949555892B11F40E94512F2091AF2AF2
:108D90003091B02AC90165E270E00E949555892B97
:108DA00009F085C34DED5CE26AEC7CE282E090E084
:108DB0000E945E08182F8823B1F18091D12C9091E8
:108DC000D22C0297029778F58091D02C882301F15C
:108DD0002092212830922228209223283092242881
:108DE0002092252830922628209227283092282861
:108DF0002092292830922A2820922B2830922C2841
:108E000020922D2830922E2820922F283092302820
:108E100080914B28882309F497C26FEF7FEF82E09F
:108E200090E00E9423084AEC5CE26DED7CE290E069
:108E300080E00E945E08882309F4ADC68091E42C8E
:108E40009091E52C0297029778F58091E32C882386
:108E500001F110926F2A1092702A1092712A1092CA
:108E6000722A1092732A1092742A1092752A109204
:108E7000762A1092772A1092782A1092792A1092E4
:108E80007A2A10927B2A10927C2A10927D2A1092C4
:108E90007E2A80914B28882309F45DC26FEF7FEF13
:108EA00081E090E00E94230880913728882309F40C
:108EB00059C20E9417086093A82A7093A92A809328
:108EC000AA2A9093AB2A8091A72A882309F44AC240
:108ED00080E00E94502B50C985010430110509F42F
:108EE00090C058018FEFA81AB80AD4012D913D9176
:108EF0004D915D914D012BAB3CAB4DAB5EABCA01CF
:108F0000B9010E9464529B01AC01C701B6010E94E5
:108F1000B55187FFE1CFAA0CBB1CAA0CBB1CE1E03A
:108F2000F0E0EC0FFD1FEA0DFB1D408051806280D8
:108F300073805801AA0CBB1CAA0CBB1CE1E0F0E03A
:108F4000EC0FFD1FAE0EBF1ED5016D917D918D9171
:108F50009C910E9464520E942C526BA77CA78DA703
:108F60009EA7D50154960D911D912D913C91579737
:108F70000BAF1CAF2DAF3EAFC301B2010E946452D4
:108F80000E942C524B015C010BA51CA52DA53EA5F2
:108F9000801A910AA20AB30A8FAA98AEA9AEBAAEF5
:108FA000C701B6010E942C528BAC9CACADACBEACE0
:108FB000681979098A099B092FA938AD49AD5AADBD
:108FC0000E9479552BA93CA94DA95EA928193909F8
:108FD0004A095B090E94B4508BA49CA4ADA4BEA412
:108FE000820E931EA41EB51E8BA69CA6ADA6BEA681
:108FF000481459046A047B0424F44BA65CA66DA6AD
:109000007EA66BA57CA58DA59EA50E946452AFA4EB
:10901000B8A806EFA01603E0B00608F4AFC060934E
:10902000AA2C7093AB2C8093AC2C9093AD2C0E9407
:109030002C5220914728309148282617370709F4E9
:109040006BC1609347287093482880934928909378
:109050004A280E9464526FA778AB89AB9AAB809084
:10906000312890903228A0903328B09034288BAAD1
:109070009CAAADAABEAA9B01AC0160EC71EE84E68D
:109080009CE40E94BA51A50194010E94715320E012
:1090900030E044EB52E40E94BA510E942E540E94E8
:1090A00033526B017C010091442C1091452CD80166
:1090B0008C918E7F8C938C918670823009F4ABC03A
:1090C000843009F464C0811169C054E0CC0CDD1C0B
:1090D000EE1CFF1C5A95D1F761C0BEE18B2E912C7E
:1090E000A12CB12C8BA69CA6ADA6BEA68ACFC7018B
:1090F000B6010E942C529B01AC0125503109410957
:109100005109A4E5B1E00E94D35027EF33E040E0DD
:1091100050E00E94B450CA01B901675E7F4F8F4F83
:109120009F4F0E9464526B017C0120E030E040EFD1
:1091300051E40E946C5318169CF420E030E044EB9C
:1091400053E4C701B6010E94B55187FF10C0C701A3
:10915000B6010E942C526BA77CA78DA79EA751CF6A
:10916000C12CD12CF0EFEF2EF1E4FF2EF0CFC12C6B
:10917000D12CE4EBEE2EE3E4FE2EE9CFAB01BC01F3
:1091800086EA9CE20E940F1D0E949F5250CF72E01F
:10919000F694E794D794C7947A95D1F7812C912CC3
:1091A0005401A3948092522C9092532CA092542C50
:1091B000B092552C9701442755272093462C309385
:1091C000472C4093482C5093492CC701B60188275F
:1091D000992760934A2C70934B2C80934C2C90933E
:1091E0004D2C2115310541055105A9F12401350109
:1091F000A1E04A1A510861087108613071058105C2
:10920000910589F4C701B601A30192010E9417518B
:1092100053014201EBCF63E0CC0CDD1CEE1CFF1CC4
:109220006A95D1F7BBCF8092522C9092532CA0928A
:10923000542CB092552C2093462C3093472C4093BD
:10924000482C5093492C60934A2C70934B2C80935C
:109250004C2C90934D2C8091522C9091532CA0919A
:10926000542CB091552C0197A109B1098093522C2F
:109270009093532CA093542CB093552C40914A2C8E
:1092800050914B2C60914C2C70914D2C41155105F7
:109290006105710561F041505109610971094093FF
:1092A0004A2C50934B2C60934C2C70934D2C409136
:1092B000462C5091472C6091482C7091492C40933A
:1092C0004E2C50934F2C6093502C7093512C452B67
:1092D000462B472B21F480914A2C90914B2CF8017E
:1092E0008487958712861386808181608083809130
:1092F000452890914628892B79F42BA93CA94DA9A2
:109300005EA96FA578A989A99AA90E94BA510E945D
:109310002C5240E00E94A62180913728882309F42E
:1093200029CD0E9417086093A82A7093A92A8093D8
:10933000AA2A9093AB2A8091A72A882309F41ACDF0
:1093400080E00E94502B16CD50E040E061E081E0CB
:109350000E94092268CD50E040E061E081E00E9477
:109360008722A2CD61E08091D12C9091D22C0197DF
:1093700009F460E083E00E94EF0461E08091E42C56
:109380009091E52C019709F460E081E00E94EF04E0
:109390008091D12C9091D22C0297029738F0809135
:1093A000E42C9091E52C0297029750F58091832A46
:1093B0009091842A8093812A9093822A8091D12C43
:1093C0009091D22C0297029740F48AEC9CE20E9482
:1093D0007E1A682F83E00E94EF048091E42C909124
:1093E000E52C0297029710F00C94BC408DED9CE2A6
:1093F0000E947E1A682F81E00E94EF040C94BC400A
:1094000080914B28882309F446C080915C28909174
:109410005D28A0915E28B0915F28892B8A2B8B2B29
:1094200051F40E94170860935C2870935D28809324
:109430005E2890935F2881E0809362288091D12CF0
:109440009091D22C0297029770F08091D32C90913A
:10945000D42C0297029738F480914B28882309F185
:1094600081E08093802A8091E42C9091E52C0297F2
:10947000029708F4A3CF8091E62C9091E72C0297F5
:10948000029708F09BCF80914B28882369F081E0F8
:1094900080937F2A93CF81E00E9421230E94E820BD
:1094A000CDCF0E94C92ADFCF0E94DA2A87CFC90117
:1094B00065E370E00E949555892BC9F480915C2882
:1094C00090915D28A0915E28B0915F28892B8A2B0E
:1094D0008B2B69F00E94170820915C2830915D2841
:1094E000621B730B6D32714014F00E94B4238091A3
:1094F000AE2A811135C11FA68091AF2A9091B02A62
:1095000060E177E20E949555892BA9F480914B2860
:10951000882309F4B4C18091F02C9091F12CA09192
:10952000F22CB091F32C8093A82A9093A92AA093AF
:10953000AA2AB093AB2A8091A72A882309F4E3C012
:109540008091A32A9091A42AA091A52AB091A62A3D
:109550004091F02C5091F12C6091F22C7091F32CF1
:10956000481B590B6A0B7B0B4F3151056105710587
:1095700008F4C9C04E96A11DB11D8093A32A9093F3
:10958000A42AA093A52AB093A62A809137288823DD
:1095900009F4B9C06091952A7091962A072E000CA3
:1095A000880B990B0E9464526B017C016091CE2D57
:1095B0007091CF2D072E000C880B990B0E946452DE
:1095C0009B01AC01C701B6010E94BA512B013C01BD
:1095D00020911D2830911E2840911F28509120284D
:1095E0000E94DE534B015C010091932A1091942A52
:1095F000C0908F2AD090902AE0901B28F0901C28D1
:1096000060918D2A70918E2A6C197D09072E000CAD
:10961000880B990B0E946452A30192010E9471531E
:109620002B013C01B601DD0C880B990B0E946452A2
:109630009B01AC01C301B2010E9449510E942C520E
:109640002B016091912A7091922A601B710B072E59
:10965000000C880B990B0E946452A50194010E9492
:1096600071534B015C01B801110F880B990B0E94DB
:1096700064529B01AC01C501B4010E9449510E9492
:109680002C5240918B2A50918C2AE091892AF0919A
:109690008A2A82019B01BF0184EC9DE20E944C1842
:1096A0008091192890911A282091952A3091962A14
:1096B000280F391F2093952A3093962A4091CE2D5A
:1096C0005091CF2D840F951F82179307E4F480915A
:1096D000872A9091882A01962091852A3091862A9E
:1096E0002F5F3F4F2093852A3093862A64E070E0F5
:1096F0000E9495558093872A9093882A80913728D5
:1097000081110E94BC318091AE2A10E000E08823D4
:1097100009F4E4C0E091AC2AF091AD2A628587E0BB
:109720000E94EF048091AC2A9091AD2ADC011A9638
:109730002C91222319F08FA48110C8C090E080E002
:109740000E949E208091A22A811104C090E080E0B6
:109750000E94A61F81E08093A22A0FEF1FEFBEC0D8
:109760000091AC2A1091AD2A0E9417082B013C01F0
:10977000D80114968C9130E020E08B3218F40E94CE
:10978000EF069C0191E02130310509F490E0F801E9
:10979000928786810E9496072FEF33E0281B390BB2
:1097A000D80118962D933C9319971A968C901A9776
:1097B0008FA6811015C01F961D921D921D921C929E
:1097C00052978FEF9FEF53968D939C9354971D96CE
:1097D0008D939C931E9718961D921C9219978CCE70
:1097E000F80187859089A189B289892B8A2B8B2BD7
:1097F00021F44786508A618A728AF801E384F484EE
:10980000E586F686C8010E940A24D8011B968D932E
:109810009C931C971F964D915D916D917C915297F1
:10982000411551056105710509F465CE441A550AC3
:10983000660A770A55962D913C915697032E000C97
:10984000440B550B241535054605570508F053CE36
:1098500053962D913C918217930709F44CCEE8164C
:10986000F90609F048CEF8011786108A118A128A83
:10987000E38AF48A8FEF9FEF858796873DCE8091AC
:109880003728882309F457CE8091A72A811158CE12
:109890000E9417080091A82A1091A92A2091AA2AAB
:1098A0003091AB2A601B710B820B930B613E7349A5
:1098B0008440910508F427CF81E08093A72A70E0C7
:1098C00060E084EC9DE20E94C41835CE0E940A2418
:1098D0008C0181E08093A12A1092A22A8091A02A73
:1098E000882321F01092A12A0C94BC408091BF2AB9
:1098F00081110C94BC4080914B2881110AC0809149
:10990000AE2A811106C080919F2A882311F40C94FD
:10991000BC408091A12A8823E9F080919E2A882367
:1099200031F060E085E00E94EF0410929E2A1092D0
:10993000A12A81E080939D2A80919F2A882309F49F
:109940005BC060E080913528909136280E944520C8
:109950000E94B4236091472870914828809149283B
:1099600090914A2822E030E040E050E00E94B4505C
:10997000CA01B9010E9464522091312830913228E5
:1099800040913328509134280E94BA5120E030E4AD
:109990004CE955E40E946C5308EC10E087FF02C0CC
:1099A00008E512E080919D2A882311F40C94BC40B4
:1099B0000E94B807AB01BC01C801110FAA0BBB0B79
:1099C0000091992A10919A2A20919B2A30919C2AE1
:1099D000800F911FA21FB31F481759076A077B0703
:1099E00010F40C94BC4010929D2A70E060E080E17D
:1099F0000E94A8060C94BC40D090AE2ADD2019F03D
:109A000060E0C801A3CFE0903E28F0903F2880910D
:109A1000972A9091982A01978093972A9093982A51
:109A20000091402810914128181619060CF455C0D1
:109A300080913C2890913D288330910509F479C0AC
:109A4000A8F4009140281091412881309105F1F04F
:109A5000029769F100914028109141280F5F1F4F34
:109A60000E151F05ACF110E000E032C08430910506
:109A700009F475C0059771F70E94D04F892F990F8F
:109A8000990BB7010E9495558C0127C0015011090F
:109A9000C701019717FD03C00E151F050CF08C01BF
:109AA000DD24D39480179107C1F0D12C16C080918A
:109AB0004228882391F10F5F1F4F17FF31C081E0CB
:109AC0008093422810E000E0D0904228DD2029F069
:109AD000DD24D3940115110541F76D2DC8010E94B5
:109AE00045208091972A9091982A181619060CF40F
:109AF0002FCF8091D12C9091D22C0197029708F012
:109B000047C0000F111FF801EF5DF74D8081918173
:109B10008093972A9093982A1BCF01501109CDCF9B
:109B20000E151F058CF28701015011091092422871
:109B3000CBCF01E0E016F10409F495CF80914028E5
:109B4000909141288C010E5F1F4F0E151F050CF4DC
:109B5000BFCF8C010095109501701127B9CF80916E
:109B60004328909144280196B7010E94955580930F
:109B7000432890934428FC01EE0FFF1FE45BF74D50
:109B800000811181DD24D394892B09F4A6CF8DCFD8
:109B900081E090E0BDCF111187C910CCCF93DF9346
:109BA000DC012D91FB013191EC013883EB0128831D
:109BB00041505109CD01BF01141615068CF3DF91F8
:109BC000CF910895B0E0A0E0E8EEFDE40C94F050F1
:109BD0006C01D62FC72F8A017901F9010995B801C7
:109BE00097FF15C08D2F9C2FF701099597FD08C091
:109BF000B801C601F701099597FD16C0DC2DCD2DE2
:109C00008D2F9C2FCDB7DEB7E8E00C9409518D2F36
:109C10009C2FF70109951816190694F3B801C6018F
:109C2000F701099597FDEACFD02FC12FE9CFA8E022
:109C3000B0E0EDE1FEE40C94E6508C014F835887D0
:109C400059019A013195219531092D833E836F8009
:109C50007884600E711E6730710578F58F81988564
:109C6000689F6001699FD00C789FD00C1124C00EB2
:109C7000D11E6C147D0420F02896E2E10C94FF5074
:109C8000730113C047012F813885821A930AB701E7
:109C9000C401F50109951816190654F44F81588529
:109CA000B401C7010E94CE4D74010E151F0550F37B
:109CB000EF81F8856E0E7F1EDCCFCB0196958795E0
:109CC0002F813885829F6001839FD00C929FD00C9A
:109CD0001124C00ED11ECB010197829F1001839FDA
:109CE000300C929F300C11247801E20CF31C673089
:109CF000710509F442C0C701280169327105B0F14C
:109D000083E0769567958A95E1F7629F4001639FAE
:109D1000900C729F900C1124C401880F991F8983A5
:109D20009A83AC01400F511FB801680D791D950150
:109D3000C8010E94E24D2C01A601480D591D9194C5
:109D4000819491089501B601C601880D991D0E9464
:109D5000E24D6C01B701680D791D9501A701C7019E
:109D6000E981FA818E1B9F0B0E94E24D9501AC01A7
:109D7000B601C2010E94E24D6C014F815885B601C7
:109D8000C8010E94CE4D43016301270119821A8246
:109D9000EC14FD0408F446C0B801C601F5010995AC
:109DA0001816190654F1892B71F44F815885B601A4
:109DB000C3010E94CE4D2F813885620E731E81E053
:109DC00090E089839A83EF81F885CE0EDF1EE0CF85
:109DD000892B71F44F815885B201C7010E94CE4D85
:109DE0002D813E81420E531E81E090E089839A834B
:109DF000EB80FC80EC14FD04A8F0B801C701F5016C
:109E000009952D813E812E0D3F1D2B833C8397FFAD
:109E1000DFCF4F815885B701C6010E94CE4DEB8040
:109E2000FC80CDCFEF81F8852E0E3F1E200E311E17
:109E300029813A81232B09F58214930408F01CCF61
:109E4000740113C06701EF81F885CE1ADF0AB701EC
:109E5000C601F50109951816190654F44F81588565
:109E6000B601C7010E94CE4D76010E151F0550F3B5
:109E70008F819885880E991EDFCF46018618970836
:109E8000A301401B510B841695060CF4A401141673
:109E9000150634F4B601641B750BC8010E94CE4D43
:109EA00092012E193F097901A101441955098F81A9
:109EB0009885481B590B2417350708F4A901141677
:109EC000150634F4B101641B750BC6010E94CE4D1A
:109ED000EF81F885E815F90548F4C401BF010E9437
:109EE000A0509501AF01C8010E94174E2F813885FF
:109EF0002E153F0508F0C0CE81010E191F09C701BC
:109F0000B9010E94A050A3CE8F929F92AF92BF92B0
:109F1000CF92DF92EF92FF92CF93DF93EC016881B3
:109F200079818A819B81611571058105910521F4F3
:109F300064E279ED8BE597E02DE133EF41E050E00D
:109F40000E94B45049015A019B01AC01A7EAB1E457
:109F50000E94D3506B017C01ACEEB4EFA5019401DB
:109F60000E94E150DC01CB018C0D9D1DAE1DBF1D7B
:109F7000B7FF03C00197A109B04888839983AA83DA
:109F8000BB839F77DF91CF91FF90EF90DF90CF90D1
:109F9000BF90AF909F908F9008950E94844F089536
:109FA00087E698E20E94844F0895B0E0A0E0809395
:109FB000672890936828A0936928B0936A28089529
:109FC0008F929F92AF92BF92CF92DF92EF92FF92C9
:109FD000CF93DF93EC01688179818A819B81611540
:109FE00071058105910521F464E279ED8BE597E037
:109FF0002DE133EF41E050E00E94B45049015A0195
:10A000009B01AC01A7EAB1E40E94D3506B017C0133
:10A01000ACEEB4EFA50194010E94E150C60ED71E2C
:10A02000E81EF91EF7FE06C081E0C81AD108E10853
:10A0300080E8F80AC882D982EA82FB82C701B601A9
:10A040009F77DF91CF91FF90EF90DF90CF90BF90FF
:10A05000AF909F908F9008958F929F92AF92BF92F2
:10A06000CF92DF92EF92FF9260916B2870916C28F3
:10A0700080916D2890916E2861157105810591057B
:10A0800021F464E279ED8BE597E02DE133EF41E0D7
:10A0900050E00E94B45049015A019B01AC01A7EA6B
:10A0A000B1E40E94D3506B017C01ACEEB4EFA5018A
:10A0B00094010E94E150C60ED71EE81EF91EF7FE5D
:10A0C00006C081E0C81AD108E10880E8F80AC09209
:10A0D0006B28D0926C28E0926D28F0926E28C70110
:10A0E000B6019F77FF90EF90DF90CF90BF90AF9039
:10A0F0009F908F90089560936B2870936C28809345
:10A100006D2890936E28089503D080819927089533
:10A11000FC01E050FC4E0895262FAF93BF93E0E082
:10A12000F0E1328131FDFDCFDC01A050BC4E2C931B
:10A130002DE924BF23E020830196BF91AF910895BC
:10A14000AA1BBB1B51E107C0AA1FBB1FA617B7075D
:10A1500010F0A61BB70B881F991F5A95A9F7809579
:10A160009095BC01CD010895052E97FB1EF4009437
:10A170000E94CB5057FD07D00E94175107FC03D017
:10A180004EF40C94CB5050954095309521953F4F0F
:10A190004F4F5F4F089590958095709561957F4FD3
:10A1A0008F4F9F4F08950E943951A59F900DB49FE6
:10A1B000900DA49F800D911D11240895B7FF0C945C
:10A1C000D3500E94D350821B930B08952F923F923D
:10A1D0004F925F926F927F928F929F92AF92BF92B7
:10A1E000CF92DF92EF92FF920F931F93CF93DF9363
:10A1F000CDB7DEB7CA1BDB0BCDBFDEBF09942A8803
:10A20000398848885F846E847D848C849B84AA848A
:10A21000B984C884DF80EE80FD800C811B81AA8117
:10A22000B981CE0FD11DCDBFDEBFED010895A1E2F2
:10A230001A2EAA1BBB1BFD010DC0AA1FBB1FEE1FC0
:10A24000FF1FA217B307E407F50720F0A21BB30B0B
:10A25000E40BF50B661F771F881F991F1A9469F787
:10A2600060957095809590959B01AC01BD01CF01E3
:10A270000895A29FB001B39FC001A39F700D811DDF
:10A280001124911DB29F700D811D1124911D0895FF
:10A290005058BB27AA270E9460510C941A530E9461
:10A2A0000C5338F00E94135320F039F49F3F19F4F7
:10A2B00026F40C9409530EF4E095E7FB0C94DA5263
:10A2C000E92F0E942B5358F3BA17620773078407CC
:10A2D000950720F079F4A6F50C9465530EF4E095FB
:10A2E0000B2EBA2FA02D0B01B90190010C01CA0150
:10A2F000A0011124FF27591B99F0593F50F4503EFB
:10A3000068F11A16F040A22F232F342F4427585FEC
:10A31000F3CF469537952795A795F0405395C9F704
:10A320007EF41F16BA0B620B730B840BBAF09150BC
:10A33000A1F0FF0FBB1F661F771F881FC2F70EC05B
:10A34000BA0F621F731F841F48F48795779567952E
:10A35000B795F7959E3F08F0B0CF9395880F08F01A
:10A360009927EE0F9795879508950E94B65208F4A5
:10A3700081E008950E94CE510C941A530E94135309
:10A3800058F00E940C5340F029F45F3F29F00C94E0
:10A39000DA5251110C9466530C9409530E942B53BA
:10A3A00068F39923B1F3552391F3951B550BBB2704
:10A3B000AA2762177307840738F09F5F5F4F220F49
:10A3C000331F441FAA1FA9F335D00E2E3AF0E0E840
:10A3D00032D091505040E695001CCAF72BD0FE2F8A
:10A3E00029D0660F771F881FBB1F2617370748071E
:10A3F000AB07B0E809F0BB0B802DBF01FF279358D6
:10A400005F4F3AF09E3F510578F00C94DA520C946D
:10A4100066535F3FE4F3983ED4F38695779567954E
:10A42000B795F7959F5FC9F7880F911D969587950A
:10A4300097F90895E1E0660F771F881FBB1F621729
:10A4400073078407BA0720F0621B730B840BBA0BE7
:10A45000EE1F88F7E09508950E9433526894B11179
:10A460000C94665308950E94335388F09F5798F0D8
:10A47000B92F9927B751B0F0E1F0660F771F881F09
:10A48000991F1AF0BA95C9F714C0B13091F00E9423
:10A490006553B1E008950C946553672F782F882792
:10A4A000B85F39F0B93FCCF3869577956795B3954A
:10A4B000D9F73EF490958095709561957F4F8F4FB9
:10A4C0009F4F0895E89409C097FB3EF490958095BE
:10A4D000709561957F4F8F4F9F4F9923A9F0F92F6A
:10A4E00096E9BB279395F695879577956795B795E8
:10A4F000F111F8CFFAF4BB0F11F460FF1BC06F5FCE
:10A500007F4F8F4F9F4F16C0882311F096E911C0DF
:10A51000772321F09EE8872F762F05C0662371F000
:10A5200096E8862F70E060E02AF09A95660F771F14
:10A53000881FDAF7880F9695879597F908950E94F6
:10A540004D5390F09F3748F4911116F00C946653D8
:10A5500060E070E080E89FEB089526F41B16611D13
:10A56000711D811D0C94E0520C94FB52990F000850
:10A57000550FAA0BE0E8FEEF16161706E807F907D5
:10A58000C0F012161306E407F50798F0621B730B70
:10A59000840B950B39F40A2661F0232B242B252BF1
:10A5A00021F408950A2609F4A140A6958FEF811D94
:10A5B000811D089597F99F6780E870E060E0089535
:10A5C000882371F4772321F09850872B762F07C0CA
:10A5D000662311F499270DC09051862B70E060E03E
:10A5E0002AF09A95660F771F881FDAF7880F9695DD
:10A5F000879597F908959F3F31F0915020F4879502
:10A6000077956795B795880F911D9695879597F9DA
:10A6100008959FEF80EC089500240A9416161706FB
:10A6200018060906089500240A9412161306140643
:10A6300005060895092E0394000C11F4882352F0A6
:10A64000BB0F40F4BF2B11F460FF04C06F5F7F4F5E
:10A650008F4F9F4F089557FD9058440F551F59F045
:10A660005F3F71F04795880F97FB991F61F09F3FFF
:10A6700079F087950895121613061406551FF2CF28
:10A680004695F1DF08C0161617061806991FF1CF78
:10A69000869571056105089408950E943353A0F0D2
:10A6A000BEE7B91788F4BB279F3860F41616B11DB2
:10A6B000672F782F8827985FF7CF869577956795CE
:10A6C000B11D93959639C8F30895E894BB27662782
:10A6D0007727CB0197F908950E94B65208F48FEFBF
:10A6E00008950E9484530C941A530E940C5338F01E
:10A6F0000E94135320F0952311F00C94DA520C941D
:10A70000095311240C9466530E942B5370F3959FA8
:10A71000C1F3950F50E0551F629FF001729FBB2758
:10A72000F00DB11D639FAA27F00DB11DAA1F649FF4
:10A730006627B00DA11D661F829F2227B00DA11DA7
:10A74000621F739FB00DA11D621F839FA00D611D2D
:10A75000221F749F3327A00D611D231F849F600D4E
:10A76000211D822F762F6A2F11249F5750409AF077
:10A77000F1F088234AF0EE0FFF1FBB1F661F771F03
:10A78000881F91505040A9F79E3F510580F00C94CE
:10A79000DA520C9466535F3FE4F3983ED4F3869507
:10A7A00077956795B795F795E7959F5FC1F7FE2B6E
:10A7B000880F911D9695879597F90895FA01EE0FE8
:10A7C000FF1F309621053105A1F16115710561F476
:10A7D0008038BFE39B0749F168949038810561F0A8
:10A7E0008038BFEF9B0741F099234AF5FF3FE10511
:10A7F0003105210519F1E8940894E795D901AA23B8
:10A8000029F4AB2FBE2FF85FD0F310C0FF5F70F4B8
:10A81000A695E0F7F73950F019F0FF3A38F49F7732
:10A820009F930DD00F9007FC9058089546F00C941C
:10A83000095360E070E080E89FE308954FE79F7759
:10A840005F934F933F932F930E94FD542F913F911D
:10A850004F915F910E9471530C945A540E9433534C
:10A86000E8F09E37E8F09639B8F49E3848F4672F40
:10A87000782F8827985FF9CF869577956795939578
:10A880009539D0F3B62FB1706B0F711D811D20F477
:10A8900087957795679593950C94E0520C94FB52AD
:10A8A0000C94665329F416F00C94DA520C94655308
:10A8B0000C9409530E943353A8F39638A0F707F875
:10A8C0000F92E8942BE33AEA48EB5FE70E94875344
:10A8D0000F920F920F924DB75EB70F920E9445559F
:10A8E000E0EAF0E00E948C544F915F91EF91FF916C
:10A8F000E595EE1FFF1F49F0FE57E0684427EE0F75
:10A90000441FFA95E1F74195550B0E94BF540F90F3
:10A9100007FE0C94B3540895DF93CF931F930F93C6
:10A92000FF92EF92DF927B018C01689406C0DA2ED1
:10A93000EF010E948453FE01E894A5912591359181
:10A9400045915591A6F3EF010E946051FE019701D8
:10A95000A801DA9469F7DF90EF90FF900F911F91B3
:10A96000CF91DF9108959B01AC0160E070E080E839
:10A970009FE30C94BA510C94DA520C94FB520E944F
:10A980003353D8F39923C9F3940F511DA3F3915076
:10A99000504094F059F0882332F0660F771F881FDB
:10A9A00091505040C1F79E3F51052CF7880F911DE3
:10A9B0009695879597F908955F3FACF0983E9CF087
:10A9C000BB27869577956795B79508F4B160939501
:10A9D000C1F7BB0F58F711F460FFE8CF6F5F7F4FEF
:10A9E0008F4F9F4FE3CF0C94665316F00C94FB529D
:10A9F0000C94095368940C94DA520E943353A8F3D0
:10AA00009923C1F3AEF3DF93CF931F930F93FF927C
:10AA1000C92FDD2788232AF02197660F771F881F0B
:10AA2000DAF720E030E040E85FEB9FE3883920F080
:10AA3000803E38F021968F770E944951E8ECF0E093
:10AA400004C00E944951E5EFF0E00E948C548B0154
:10AA5000BE01EC01FB2E6F5771097595771F880BAE
:10AA6000990B0E94645228E132E741E35FE30E94C0
:10AA70008453AF2D9801AE01FF900F911F91CF919C
:10AA8000DF910E9460510C941A53FA01DC01AA0F65
:10AA9000BB1F9B01AC01BF5728F422273327442753
:10AAA000507820C0B75190F4AB2F002446953795CD
:10AAB0002795011CA395D2F3002071F0220F331FBC
:10AAC000441FB395DAF30ED00C94485161307105F0
:10AAD000A0E88A07B94630F49B01AC0166277727C6
:10AAE00088279078309621F02083318342835383E6
:10AAF0000895DB018F939F930E94D350BF91AF9134
:10AB0000A29F800D911DA39F900DB29F900D1124C7
:10AB10000895991B79E004C0991F961708F0961BB9
:10AB2000881F7A95C9F78095089597FB072E16F42C
:10AB3000009407D077FD09D00E94A05007FC05D0F3
:10AB40003EF4909581959F4F0895709561957F4F44
:10AB50000895EE0FFF1F0590F491E02D09940E94D7
:10AB60003951332312F48A1B9B0B0C94B9550E9464
:10AB70003951B7FF0895821B930B089597FD1094E8
:10AB8000002E083098F00850232F342F452F562FD1
:10AB9000672F782F892F912DF4CF1594979587954E
:10ABA0007795679557954795379527950A95AAF70D
:10ABB0001124002D08950024A7FD00942A173005C4
:10ABC00040055005600570058005900508950F93B8
:10ABD0001F93CF93DF938230910510F482E090E0D1
:10ABE000E091122EF091132E30E020E0B0E0A0E0D2
:10ABF000309799F42115310509F44AC0281B390B07
:10AC000024303105D8F58A819B816115710589F160
:10AC1000FB0182839383FE0111C040815181028137
:10AC2000138148175907E0F04817590799F410970E
:10AC300061F012960C93129713961C933296CF01E3
:10AC4000DF91CF911F910F9108950093122E1093D1
:10AC5000132EF4CF2115310551F04217530738F068
:10AC6000A901DB019A01BD01DF01F801C1CFEF01AC
:10AC7000F9CF8093122E9093132ECDCFFE01E20FC9
:10AC8000F31F819391932250310928833983D7CFC1
:10AC90002091102E3091112E232B41F420917128F8
:10ACA000309172282093102E3093112E20916F280E
:10ACB000309170282115310541F42DB73EB74091F0
:10ACC000732850917428241B350BE091102EF091BD
:10ACD000112EE217F307A0F42E1B3F0B281739079C
:10ACE00078F0AC014E5F5F4F2417350748F04E0FE8
:10ACF0005F1F4093102E5093112E819391939FCFFD
:10AD0000F0E0E0E09CCFCF93DF930097E9F0FC0107
:10AD1000329712821382A091122EB091132EED0160
:10AD200030E020E01097A1F420813181820F931F41
:10AD30002091102E3091112E2817390709F061C08B
:10AD4000E093102EF093112EDF91CF910895EA0138
:10AD5000CE17DF07E8F54A815B819E014115510559
:10AD6000B1F7E901EA83FB8349915991C40FD51FDB
:10AD7000EC17FD0761F4808191810296840F951F85
:10AD8000E90188839983828193818A839B83F0E0A0
:10AD9000E0E012968D919C9113970097B9F52D9153
:10ADA0003C911197CD010296820F931F2091102E96
:10ADB0003091112E2817390739F6309751F5109236
:10ADC000122E1092132EA093102EB093112EBCCFE2
:10ADD000C283D38340815181840F951FC817D9073F
:10ADE00061F44E5F5F4F88819981480F591F4083FE
:10ADF00051838A819B81828393832115310509F0D8
:10AE0000B0CFE093122EF093132E9ECFFD01DC0104
:10AE1000C0CF12821382D7CF81E090E0F8940C94D7
:06AE20001157F894FFCF6A
:10AE26000100010001000100010001000100010014
:10AE3600F3F0F6F0FAF0FFF003F17BF112F115F101
:10AE460018F11BF11EF107F109F165F00BF10EF196
:10AE560011F114F117F11AF11DF100000000800143
:10AE660000000003000080030000000400001E0034
:10AE760000007A00000072010000E8030000881359
:10AE860000000000FFFF0100FFFF02000300FFFFBC
:10AE96000400FFFF05000600070018000C0006006E
:10AEA6000100FFFF0200FFFF03000400FFFF050093
:10AEB600FFFF06000700080000000000300A2C0A09
:10AEC60000093D90D00380841E90D00324F4000036
:10AED60024F440420F00127A40420F90D003000043
:10AEE60000000000803F0000A040030201000C0D9E
:10AEF600040500000003000102000001010000003B
:10AF060000000000000000000000000032F139F1EE
:10AF160041F148F151F159F160F168F172F17DF1B9
:10AF260005040005060204010300010001020302F4
:10AF36000100020304050203050400000000D20517
:10AF4600160937052306680546055A05751A1E07AC
:10AF56007405A109000000003E0A782A8E0A5F0ADD
:10AF66003F0A920B410B9E29980AE20BDC0B5D28E7
:10AF7600D40B00000000600D3B0D721A110D340D4C
:10AF8600210D120D310EEC0DDF0DDB0DA20D830D23
:10AF96007B0DB10DA90DEA0CE50C20100120400433
:10AFA600100208010201020408040201040810202C
:10AFB6000408201002020005020105000401010434
:10AFC6000404030303030505030300000101000055
:10AFD60000001B171609721A711A3411D814951429
:10AFE6002C14AB13EC13C719C714B3101711C912DD
:10AFF6003A13B812C4184C18ED17B328A90F2B0032
:10B00600202000202030006F666600536574200003
:10B01600536574207377696E6720002D002A004DF2
:10B02600756C74697374657073004D6963726F74BF
:10B03600696D696E6773005B005D0053657420730C
:10B04600746570733A0053746570203120736574AB
:10B05600004446414D205468696E670076312E39AA
:10B0660000436F6E66696775726174696F6E00532F
:10B07600637265656E73617665723A00436F6C6FD5
:10B0860075723A00416C6C6F7720666173743A0092
:10B09600496E76657274204C43443A005050514EC6
:10B0A6003A004D4944492063683A0043616C69623D
:10B0B6007261746500506C6179204332004F4B20F9
:10B0C60028002900506C6179204334004F4B00441E
:10B0D6006F6E65004661696C656400536574207324
:10B0E600746570733A200042504D3A20004F6E004E
:10B0F6004F666600426C75650052656400416C6C73
:10B106000037003800313000313100313200313340
:10B1160000313400313500313600496E742E004559
:10B1260078742E004D494449003234004E6F726DDA
:10B13600616C005265766572736500426F756E6369
:10B1460065004F64642F4576656E005368756666C4
:10B156006C650052616E646F6D004356204D6F64DE
:10B1660065004D494449204D6F6465005365742060
:0DB17600737465702031005377696E6700B7
:10B183001027FFFFFFFF3C028B01182FF111F11E67
:10B19300F10024F400015A00010200FFFF000080C7
:10B1A3003F01000100010001000100010001000155
:10B1B300000000803FFFFF0100004843000008003B
:10B1C3000000010000000078000000000000010002
:10B1D3000200030004000500060007000000000051
:10B1E300000000FFFFFFFF0100000001000000005E
:06B1F30000142E80000094
:00000001FF
